:100000000C94E7000C940F010C940F010C940F0159
:100010000C9436190C940F010C940F010C940F01E1
:100020000C940F010C940F010C940F010C940F0110
:100030000C940F010C940F010C940F010C940F0100
:100040000C94BA370C940F010C944D290C94D529BB
:100050000C940F010C94041A0C940F010C940F01D2
:100060000C940F010C940F01E12E212F5E2F7C2C9C
:100070009E2FF32EED2E352FB02FE62FE62FE62FF5
:10008000922FE62F1E2F172FE62F0B2DE62F7C2FFA
:10009000E62F472C112DE62FE62FE62FE62FE62F31
:1000A000E62FE62FE62FE62FE62FE62FE62FE62FA8
:1000B000E62FE62FE72EE62FE62FE62FE62FE62F98
:1000C000962FE62FE62FE62FE62F142F7902037CDA
:1000D00002037F02038302038602038902038E0266
:1000E000069402069A0203A002039D0203A30203E0
:1000F0008C0202A70201A60201A90201A80201DDE9
:10010000025DA9135F2A8706934B122C4B8BA45CCC
:1001100048BC604A31175FAB1360CB871DEE4B12B2
:100120000F4B86225D4AC3604C89295F8E135F1195
:100130008730974B12284B868D5C4FCC604F463DE5
:10014000589D1361208740B24B175B4B88865C48F3
:10015000DD604A32565DAD13602F8759B64B1348A8
:100160004B87625D480D604AFE6B5D351361C88741
:1001700073DD4B14E44B88FE5C4A9F604F197C583A
:10018000D31361E98786C34B14014B88005C4BB8DD
:10019000604A2B915FE0135FF1879B834B143E4BCA
:1001A00086405C48DE604A53AA58E3135FF487AE8A
:1001B000F24B12E04F86545C4B93604A35BF5FF8B8
:1001C000135F4883C75CB60E8582C1F21570228228
:1001D00068431DB191F13C0852664FA9B13EFA65E2
:1001E00002B6B1F860098A7753DBBD94FA8C37A95F
:1001F0005FF10A2F36155F892EF0F5C34D59A80817
:100200006F2953EF8FA9151E6B1CF45F47A55B8404
:100210004D2D8F4EDA555719406745A59D85918B19
:100220005E493EF6511A7CC641A683E393B94F4816
:1002300021F0B68624CC38126EDBF53A4EDB7D5FBA
:100240009B1F4CCA5A1266DE15DA2F4891F1B98607
:1002500030CD2612BEDCF356DFA991F1B68650CA26
:10026000581266DE05F4914891DA5A75E0BE48D11D
:10027000E22905E03248A04DE8741CBE47A5824A39
:100280008D14DCA991F1B5860ABED9F1CD29931B55
:100290007A4819F3CB6516CD2512E829157D3AA9C0
:1002A0001FF26D86ACCBC8F1DEDCF1AAD1A6B04D51
:1002B000AD66BCCA6D1266DE05282E48A1EFBA866F
:1002C000E0CF27125EE0F6366ED8805F6C9C3EAEC3
:1002D00069A2CB4AA7F63FB91FF25A86CCCC2412AA
:1002E000DEDAF1E2CED81161D2A883AE13AB690990
:1002F000B26B7FA931F1B686F9C9D9A4CF4A056C92
:100300002E481FF25C8616CC27128B09B4527EDA77
:100310007F5F6FB554AFC9A2CA4A08E67A891FF257
:100320005C86039E6B34D739A6797EDA7F5F6BA833
:10033000E1AA64ABDEDA5B36CED8E85FD9184D5F50
:10034000C9A4D04A95857ED8E75F79169B5FC9A27C
:10035000D04A15C22D483975828C73AE47A56F4AB5
:100360000B81DEDA7F5FC916A75FC68EEEDAF16E0B
:10037000D66A3A4EDB82719E47A5904A8DE8CCB68C
:10038000131E5719C55F41A64DDB841951DA30F1B0
:1003900018184DCD59A3BD4A2276B767A33E42B384
:1003A000A7B958F11F2956478948FEEFC686207124
:1003B000C861E1794541AEA9FF6D48A45C03B7600F
:1003C000DECA1642A64843F5DA084ADD95124BDA32
:1003D00081405FD901DF29B2D1CBC1347F397DDEC5
:1003E0008ECAD1F1A88629014E6F7D9849DDBFBF25
:1003F000F0EF1816EBCF46A25DD9746B56DCE0F037
:100400002817EDCCB6A32DDC649AB2487BE5B9651C
:1004100090BED9F16CDDE42D35488D5F69652EBE47
:1004200009F1BA2C93B14B72ED5F1486A7D9D59818
:100430000BD043B43EA9813EC965A9BAEE12F44A75
:1004400093D59870ED5F1486C7D9D19C07D43FC46B
:1004500081D8E0EF4815B9CE96A12DD98DC891DA93
:10046000F0F135867FDC2194CC2993FFA1482CE85C
:10047000650F6FD4579B78CB9EFB47CF29E4281696
:100480004FCF41A66DDCA41491DA21F049864EBE0F
:1004900040F26E299D55D266A13EC9246C5FC8B05A
:1004A0004E56153CAE44228235DD5411CA92E66C9C
:1004B000CE41DFC8A3DF258655CFB5A262C97A3EFB
:1004C000BE641AF318E446CF16122660A53E91D8F2
:1004D00030EF5816DCCBC9A25E4A0DF877B91FF28F
:1004E0008B8763BEC9A45E4A8D7C51DA30F118183F
:1004F00071BEC9A45E4A451757A8213E6145727175
:10050000D9F1DEE87504DFD6016BD924FC535835E8
:100510004AA1835CDDC8998192759BDFDB923A4AE0
:1005200072B0A2D813DE3C06C87340A62DA805BE43
:100530000148D9756978F9CF56A26DDA8DA841DAEC
:10054000E0F1281854BE80F22E29988BDF66A13E78
:10055000D524A25FC4B04E5621C6AE44228235DDFA
:100560009E11CA92E66CA697DFC8A3DF5719934C79
:100570005670DEDAE474465E59512816B3CF56A29F
:1005800066DE541081DAFD5FB80EF2D3C138D5466D
:100590000504C6661FF2AABFB7DB719AA7D2DF16A1
:1005A00050DD2699571988649512294AAD2867CCE1
:1005B000936DDCA46BCF86A266DE542881DAFD5FE2
:1005C0005719035CA1924E2973C6A156F3BC46D4B9
:1005D000F0DF78928664BEDC9748F0EF1816D6CB31
:1005E00086A43DDC71E423CA7DE1D1AC9BA3C9A6FE
:1005F000F67893673F7340E3810EB3D7139A6CDDAF
:100600009A3A50DD3F982586C35FD694ECCC649E21
:1006100091D819F3781729CC06A3BDDBF48F21DB21
:10062000A0F0E8178BCCF6A32DDB64B9B1DB10F09A
:1006300058182DCD86A43DDC528E80FE3CF5583BEB
:10064000B8CA97D06D0752F8C76D733E6FB37F720B
:1006500081D1C775FC71D7A8A13EB123AC5F20AF93
:100660004E56FDFDAE44228235DD9411CA92E66CF1
:100670008E85E889945F49946941B11244567C6241
:10068000B046107D38E47811A9914FC94C8CEF48E1
:100690001FF2F4C0E4CB28A6DD98F41826CE7AE148
:1006A000C30800DEFA91234A36A850DDBC99B91A76
:1006B000D1CB3660C7D0FF3035CA8DE10D056BDE7A
:1006C0008F120F4A9351F57281F3AA1AB311CF3FDB
:1006D000D9D0F25020CADF5F4A1BBABC37F56CDDB7
:1006E00063D7D66A1A52A945EA005460564AC56FC4
:1006F0000FC90BE032074ADCE2933CCB527F9048B3
:1007000012F4A9677ABA47A53C7F0D2857BD5D1E34
:10071000418672DF3892C262FA10D66E885BC91ABF
:10072000B87147A5BF832026F248713EB965AEBEB9
:10073000DEF56CDD4B0C9867E88C31B3C5700F406B
:10074000B578ED6C2766DC5F03866ABE79F1074AEF
:1007500093C59C70985D4F45AFA4B9A5554175CB25
:100760005FA9121E4965A15FFF127E29B58D1EABE0
:10077000624257196565CE0E76094C7AE848313EDB
:100780007965CDB91AF56CDD47B0465F854E826C50
:1007900033707BF111772B9BE955D85FFF8690CAA8
:1007A0007A4B534AE52E5F89113E480655DDC196C6
:1007B000E8CC1E36C5CAFBE3350837DCB2965CCC04
:1007C00053C05FDF7140C769C6CA97475F79C63BB0
:1007D000AD48F8B646D457BEDC96EF5A053DDBCEA1
:1007E000A4F2C916BB5FD127663DB824D7AEA33E9D
:1007F0005719154A47A56D7A0568A24B1FF2ACAF91
:1008000010CCCE1789DF94B1A6DDEF1D5843C3E1AC
:1008100096A22DDAA48451D810EE3815C3CE86A145
:100820001DD934B3C1D9A0EEC81545CE16A1ADD996
:10083000C4A171D919F31818E7CDB5121FCA57BE54
:10084000D4C8998132758D5FE338F54625D8E466C2
:1008500054E79D0E31D73F9AE2581A44F856C87DA6
:10086000CC10F6D5EC9C14D40E46C466BC8D04ACFA
:10087000D7A3F3A682CABAF676464A7D791459D52B
:10088000E19217CA9B1373D84DEF601C2CDFF9F16E
:1008900005A142DC43DF9DEF661CFDD7C822BFDE09
:1008A00053A0A7481AF3281667CF41A62DDC643C55
:1008B000B24899E3E20ADE45301CE670FC40DEDC1B
:1008C000A98D5719A56462969ACED24E00CC1FF21C
:1008D0005EC0DCCA674BEDD20BC2C76E985BD91AFB
:1008E0006651DE30F6D8146C72C84EDFCBA07D5551
:1008F000E338F5462560E466CB8DF2B46471C13807
:10090000E9D42188F3C2CFE92816C5CF41A6E12951
:100910000582944891EF5C8697616005E429938B8A
:10092000FC7191F15C8606CFA1138EDA6E2F974889
:10093000753FB9653ACAE24CC058F8242EDAD45F44
:10094000A918805FC9A2484B15D8B54B996DE2A490
:10095000D851D030C329F5B750DDBC99B9189F5F85
:1009600029A41E4A95F7E14819F3B81713CCC6A37A
:10097000FDDB34E1E1DBF0F0381785CC46A47DDC0B
:10098000541281DA91EF5C86904845011B091438B6
:10099000A6DD71EF1686E6CF8712ED080B71CFA9A1
:1009A0001FF2398AC4CFAD13CEDA6AA9DEA9A13EFF
:1009B0006916795F79A22A4AC99E69B451F39DB438
:1009C000CECA314C094A41C6B2A987F3B01A99CBB5
:1009D0000EA648DE56220EDAD65F8918185F69A285
:1009E000464BB572B74B53759C8C46AAC9A25E4A5A
:1009F0000DD277B8923EC918475F47A5A04B056E48
:100A00009A48A1EF0E8624BECE43F05049FDDED8B1
:100A1000E05FC9ED069E69A21D4AA738DFB931EF34
:100A20000B8612CF8A128260BA2E12BD1FF2BE87C9
:100A300020CCF612DEDA5436D13E91F118861ECF64
:100A40008D128EDA4A44DCA93790818C40AA15D1E8
:100A5000DEDA6B51CED8F8608916955F6128975021
:100A600099951E2D121E980028CD86129EDA6F6D64
:100A70000ED8FC605D9B63584501A40905EC9E48B7
:100A8000A1EF0A86AC4970188A394F8A7A5E4665AA
:100A900055795B5F99A1BD4A8C7E4FA964462EB300
:100AA000F2BEBC3F1E29D1A6F46DA85AE9191472F2
:100AB00060D1564A0534D66A0A4E40866CDFB112C0
:100AC00090E0E5432FC97E8DB9654ABED9F17EDA43
:100AD0006FD36ED8FC608DACEFA309A6B278934BB0
:100AE0002672B65FDD86E8CAF74CEB78150D7652B4
:100AF0004A693C86C1DD6D942DA88CA5410619F28A
:100B00002AA1F3428426073F649891D830EF581603
:100B1000EFCEA6A13DD94487F1D9B0EED81561CE6C
:100B200026A166DEA5B4954841EF15863E485A17C2
:100B3000323D9D25474FCD52F3ACADA3E9A61878C1
:100B400081A1D646AA7DF3A4F341B3A62F40C9687C
:100B500069B451F39DB4EA5F84126CDD43666EDACA
:100B6000F6606918805C41A66EDB546ADED85B6271
:100B7000D1A86BAAC8F1DEDC5478DED8C660D916DD
:100B8000365C49A8E73D0516E94BA1EF01878EC900
:100B90001005DEDA3E97CED8CB60491CB5AAC9A2B3
:100BA0002D4A07C3DEDAE05FC916655FA40050294D
:100BB00015517FD83381BA75675FE2680E89B12E0F
:100BC0007C6A1A52CDE5195FEC680E89B15C7C6ACB
:100BD0001A52D1E54B01DA41BF400548914819F35B
:100BE000458667DFDF92C664FEE29548BB85E082FA
:100BF00050CBF3409ECAD6763CC884DFCD946B417F
:100C0000EF3015680586CFCAB3E1FC0808DE4DD188
:100C100013DE2C86C9DC98F35319C8A9DF94E3CC02
:100C20008DB4A24887E1AE08E35FE338F54625BA04
:100C3000E46615DE4D45BE51D0300868402254DDD3
:100C4000E355C908D5DDEB9411CC8DDED1DBB0F0D6
:100C5000F817EDCC86A33DDB74CBA1DB998CC918CA
:100C6000B55F89A1864D55F7774DF1EE73899ECE1C
:100C70006215C678F595DEA9A13E57191D6469FC79
:100C80009D29C66109AA1FF25EC02D5FDF126CDDCF
:100C90004BA850DD44982586535FD9A4324A050CF1
:100CA0008D48798BB96526BED9F16CDDE4977EA9B4
:100CB000413E8A6BE1BA47A57384D0BA0248D85F37
:100CC000FF86655FDF126CDD9AF274A54349946D6F
:100CD0008ABB47A5738420D6F248D65FFD86D0CA6A
:100CE0008F4A6CDDB8DF8248DC5FD9183E5FC9A44B
:100CF0002F4A0562944BA0BDC9182A5FB6A14DD9F1
:100D0000649191D9D0EEF81597CEC6A166DE749D98
:100D1000A1DB20F16818D9CD96A44A4ACD9807CC1A
:100D200019DF6206654B18167F3D863E4F4C1A52FE
:100D3000DE45D8DEB291DE296D2FD6A90964F5799A
:100D4000875F49A12E4A8787D646AA7D5319ACA949
:100D50006B389170AD4E674213755C8C70AEC928CC
:100D6000EF50A197D248121ED286EACF9C12E66CB1
:100D70008E853389DB5FE5863C797E0E9EDED95019
:100D80009448CA5F5719FE6569A22F4AB51C8C4862
:100D9000513E99659ACAA94C254A2FBCC9B4B1F3F2
:100DA00003B48A497018A850E0AE4AB9113E59659B
:100DB000785FE338F5462522E466CB8DF2B42671E0
:100DC000C1386ACAA24470C850DF519CD559631813
:100DD000995029271ED8E45F99160E5F29F1CE2974
:100DE000C5EE0F56737DBCA4A4DD1494CCCC046C6A
:100DF000DA5EA665EF8C415985017A0905EACF4E86
:100E0000B365FC8CB8AA09A2314AD59A8A48713ECA
:100E1000B96516455C1C8454BC1252CA2EE1770891
:100E20001FDD41287750AF20654E3552D508B3DD20
:100E3000E7941DCC11B4C3C8BFDF0806B571D34019
:100E400009784064F9B4CBF3E20CC2D94ED17C5D91
:100E5000A4554AB9113E596541D941983DDA54CE5D
:100E600041D820EF481589CE41A65A4A96EF4ECB7D
:100E700025E05E0762DC5E936FCF95FD56DC91EF57
:100E800014870A7D5001E6FA05EA5C89990FD801BA
:100E900018E759A317491177DEDAC95ECD651ECD73
:100EA000F511E829154550DD219659177B5F59A3A7
:100EB000344A8D26C4A5201EDAD5D3AA59A31A49CF
:100EC000A550884841EF2086E70176608EDC5CCE35
:100ED0007EDAE75F4D45F6CFF51185487212CED820
:100EE000CA5EE19CADAEC9A2344A157A894812F4B3
:100EF000D918255FC9A4344A8D6C91DAD98DCD6F8C
:100F000080CDF5111E488FC7DEA81FF2A38CCECD71
:100F1000F211E2310586E2499142524594BE47A55D
:100F2000B85045B0E5499546C918965EC1F26CDDEA
:100F3000DF3691D819F3CD6EB8CDF51166DE05AC6C
:100F4000E5499546C918FA5EC1F36CDDDF4A56DC07
:100F5000E0F111B4DC7D6001E23505C8E24991435E
:100F60004D45E6B6C9A41A490D8C50DD6B65C9160E
:100F7000CB5E8534773D199ECEDACD5E181676CBE2
:100F800086A33DDB7417A1DB20F1681843CD96A43E
:100F90005E19522480FE7B5F29154C5FB9A1354A4A
:100FA0000DAEDF297AE1C308A6CA3418C7CA8B8000
:100FB00024C8288D5645BECA88192F51065D9F5DED
:100FC000E262527944BE47A506507DCADFDAA05FCF
:100FD0000A99035AC808DF29A548884841EF2086A6
:100FE0000248BA176739050751D920EE281621CFD4
:100FF00056A26DDA8465B1D9F0EE1815F4CB86A34C
:101000003DDB849151DA30F11818D5CD46A32B0081
:1010100063A6A6677B5FD286905120946CDD021890
:1010200037C8978D5719B959C63E144A2D2C50DD33
:10103000D1655815EBCF86A27DDA94AAA1D9F0EE3E
:1010400018154ACB86A43DDC94DB93FEEF15F7869A
:101050001F0116607F29B5B750DD1065D20651CE4D
:1010600096A22DDA8DF051DA30F11818B3CD49E19E
:101070002B0063C45ED8E75F5916AD5FC120A8CCD2
:10108000EE0250DD8E65B2060E7147A5FD50CF0E03
:10109000DA661FF2E88C12B7C9A41A49067D7ED819
:1010A000E75F7916735F4B2871508E5BDEA920EEE7
:1010B00058156DCF86A27DDA942856DC20F1681889
:1010C0000FCD96A45E19945593FEEF154916185F3F
:1010D00059A2354A0DDA75CA5BE1B208D2CA341892
:1010E000C7CA0BCC50DDB06593066E7147A5FD50A5
:1010F000B070DC661FF2E88C7CB7C9A41A49061FE1
:101100007ED8E75F7916D15F4B2871508EFDDEA93E
:1011100020EE58151BCE96A22DDAA48A51D819F3C9
:101120001817FDCCA6A35DDB93BD8F7EA1F1708760
:10113000B0CD6F13BEDAD0332ED85D62D1AC49A3E7
:10114000C9A6F67893D13F73ED5F1486CCCDA71274
:10115000EEDC7452FEDA015FF918AB5F463F4E29B0
:10116000544FAEA9F08C39658770B9F15D7775423F
:101170009EDB396019175F5CA9A3884B75EF754B2F
:1011800071EF9689F4CF0715E670FC76DEDCA98D49
:101190005719F3649512294A050AAC48A1F13C8617
:1011A00000CDBD120EDC7AA69EDB3D601917835C74
:1011B000A9A38C4B7527714B71EF9889CCCF19156A
:1011C000E670FC3EDEDCA98D5719AB649512294A06
:1011D0000542A848A1F1408678CDB1120EDC7EDE32
:1011E0009EDB41601917D75CA9A3904B757F6D4BAF
:1011F000934CDD6564CD9212DEDC5FFAA1D900EE7E
:101200002815CDCE41A6E0793DF93666813EC96507
:1012100080BE47A5BF83A5F76EA951489A6910CA39
:101220005C4CF94A31243EA9813EC96DB3BD47A546
:101230002482BB1C7966151E867116B2C5F5FB2C7F
:101240005E40A666FA8D94B41A712140D778C5DC49
:101250006A4B61F17E8736CD7F13CEDCBC5FE748F9
:10126000988DDBB4CB71F7401A4A526A71AF433F95
:101270008C6528BD47A573846178954891F1818775
:1012800010CD7013FEDCBF85EEDA4C60511AA1CC94
:1012900076A3ADDBE40731DB90F0D81703CCE6A3EF
:1012A0001DDB543181DB00F04817A5CD56A42DDCA1
:1012B000642293FEEF15291CB7E8B1A53C08940100
:1012C00093F651EF9A8996CF1B15C470DC303EDC43
:1012D000878DC916E85CD9A29B4B254A604BC1EFAC
:1012E00088876651DC3004683CF6DEDA4D60D91838
:1012F000CD5CE9A49C4B3564614B51EF9C89AECF2A
:101300001D15C470DCF83EDC878DC9164C5CD9A273
:101310009F4B25821C4BC1EF8C879E51DC300468AB
:101320003C3EDEDA5160D918695CE9A4A04B35BCBB
:101330001D4B51EF9E8966CF1F15C470DCC03EDC8B
:10134000878DC916005CD9A2A34B25DA184BC1EFD3
:101350009087D651DC3004683C46DEDA5560D918F7
:10136000255CE9A4A44B35F4194BF1EF348B9EBEF8
:10137000A66A5C9805F4DF792A525719107B89D543
:10138000E7798E73958891EFD08B0E6E4005160D20
:101390008075B167053E48B330B0C33FFF291FB128
:1013A000E6AD7C8CFB65DD7067FF8F29BF2277C6B9
:1013B000934CDA652AD1C4A08A4A9EBA5DA9785FA7
:1013C0001F862FCEB4A1CB4A79C8DFD8A2EF98866A
:1013D0003850B02F314A7245A3DB4E5F3A86BFCFFB
:1013E00038A2DFDA167441481FF277BF305F8212ED
:1013F000F54AADE86742E35F7618C7CD64125F999E
:101400007EF7DED8EB5FD916D35F49A8D73A869826
:10141000CEDAEC5FC918CC5FA49E5CD6E68C2FD8E0
:101420000FED3614AC793E0EDEDE1D0450DD7298F1
:10143000736505B30AFBB92C93AD4B72AC5FF586AF
:10144000E9D3F39ECBDA02D6D3D8ADEF57191067A4
:101450009512294A6ED8A4C492F1DA18FDCDF8A4E9
:1014600058D86EEC5116148E027B209AC9A24C4AB1
:1014700015E0B148B1EF3986C8CFB812E7EC1FDCF0
:10148000F5EACD01A916CA5C39A2AB4B0DAA29B465
:1014900091F3E1B49ACA284BA94AE19ADED8075FD2
:1014A000D916555FE9A2564A3538A7489E01E72864
:1014B0001FFDF1B8BEDACDB52ED85A60D1ACC9A3A4
:1014C000C9A6F67893513F737A05C32C47F9D5B86E
:1014D000C7EAFF72D5E8ADFFEE864E5F47A573847D
:1014E000F0E022487EFFC72667FFD1B687EEBF4AED
:1014F00015EC6D035719E365D2120A4A4CFCE84813
:101500001FF2A6BED85F8212EBD0238CF1CEC9E9C0
:101510008915E05F19A1514AE589AA4881EE3E8606
:1015200040CF0313CEDAD025D66E885BC91AB671C8
:1015300047A5BF83F0342248D45FFB86995FDD1254
:101540006CDD9A7815486D5FB62634FFC6B2F6EEAC
:101550002C50C8481FF25EC0C35FE512234A395EB3
:1015600050DD6E972586AD5FC09CF8D430E6E2C2B0
:10157000D45FFB865DFB73B6A9EEE1DE50DD2699F4
:101580009486DE5F20B2D8EA1028C2E8B85FDF8612
:101590009ECA5C4CF94A31969B48C55F5719C36790
:1015A0009512294A122EC0C2C0E901148CCE7D13B7
:1015B0008ED9BAB11ED9476099158D5CC9A2964BD8
:1015C0001550674BB1EF838778CF7213EBF0236828
:1015D000F1EEC9093167B870ABF1DC7763DC43DF4A
:1015E000CB01F22805B2BBF15CEC724879AC453E08
:1015F000832CDBF949F10BD6437433D88EEF0714F3
:10160000ADD1C138D5460592C6661FF2AABFAC5F00
:10161000D8126CDD9A2EC548BD5F3212E6D32992EE
:10162000CFCA07A2CDC81FF2A7BEF65F821247D667
:101630007FBCDECAA2E1EB088BDD9A12EBD922AFA8
:10164000F3D9CDEE3226BCFF88A12FD966DDAFD904
:101650000B013228935FFF127E29B5BF12A0664AA4
:101660005719A067CE0E73094C68E848313E796976
:101670003CB71CF56CDD964C465FBD5258B38EBE30
:10168000863F4E2D64ABA2A0008C3E697370B93EBC
:10169000680994BDAEA9E08C39694570B5FA4D77FB
:1016A0007A4DA167018B10861E5F64B69CEED40A4A
:1016B00006E01FF25EC02D5FE512234A39BC50DD03
:1016C0006F97E4866F5FF512314AD25803DA7EF1E4
:1016D000C618EF5FA4B25CEA6649AFD90F0136289D
:1016E000B8710040E07818C8FB66C58D0586235F99
:1016F00047A58C8361F495489F6BE8A255FBF3B630
:10170000EBDC2290E4EEBA0558E4E3D3B39E92DF1B
:101710007F9EB7C6148E52757691BBD3E4798EEF57
:1017200017881FF21ABC06CF6F138EDAAC2FE2486F
:101730007379BC9044CD6C13BEDCA939CEDA386025
:10174000C918645CC9F1EE2993DD017331EF758925
:1017500060CF64159EDAB3530ED8406257194B65BB
:101760001F3FA5777D4BB7674F5F51190D42382D4D
:10177000EA2C0D5DDCA9A98CDC65B3709D12CBDA77
:101780000210D3D8ADEF5719E9644C3E7276B4A27B
:101790006064BA5FE18698CA5C4C3A4A509CAD4896
:1017A00092F1DA1805CDF8A49D4A59AA43DB2EF030
:1017B0006617AFCC041228DD8E4EDED9FF5FD91537
:1017C0002F5FE9A14E4A3557AF48D1EE3B861ECE7A
:1017D000BA123ED979D4AED9065FD20646DFE2927C
:1017E0001ACA0E6CC4C6BCED05146ACFBF12EEDA7D
:1017F0007CF0FED8095FF916015FC4A0FCD83470F4
:10180000E6EA9AE3E30AADDBF596E7EC1FAEF5EA0C
:10181000CD01B2126ED3C29EFAD6B29660C460EB0E
:10182000A1262CCA5C4C894AC12837E88BFFD426F4
:10183000ACFFEE12F44A93A34B72AC5FF586FD5FEA
:10184000FB126CDDE27CC548BD5F0E86F85F47A5E4
:10185000BC826152954891F13786CACDA612FEDC52
:101860007560EEDA025F960536DE2691D6CD486EBB
:10187000EC483EEB871239D311B26CDD9A4633EA5D
:101880008F01D8281CF920B2D8EA102AC2E8B65F26
:10189000DD869CCA5C4CF94A319833E88FFFD82624
:1018A00038FB47A5BC8220A6F248D85FFF86A0CAB5
:1018B000174A3A4A50B4DEDA035FD9184F5FE9A4F9
:1018C000524A3550AB48D45FFB866D5FDF126CDD4A
:1018D0009AEA35488D5FB212A2D3C29EFAD62ADEAA
:1018E000CA481FF25EC07D5FE512254A3BEC50DD21
:1018F0006F97E486585F249EDCD61476C6E81FF204
:10190000A6BEDE5F8212DEDC7B08CEDA085FE91855
:10191000E85FF9A4574AEE9A24C49CEBE5123ECF47
:10192000B7128EDA84241ED8116099162D5C47A553
:101930007384F0322248D45FFB861ACFB3128EDA5A
:1019400080401ED80D5F9916B55F47A57384204E61
:10195000F248D85FFF8658CA144AC94A015C37E882
:101960008BFFD426F8FF69A2604BB5FA5D4B51EFAF
:101970004D8722CF4C136CDD9A42C548BD5F10865F
:10198000365F47A5BC822086F24871EF9787FECF6D
:101990000613DEDAD597CED862605719C267951262
:1019A000294A0530104BA1F198870ACD19130EDC96
:1019B000D6B3F888948E5275329E69A2504AB52EDD
:1019C000AD4851EF3D8696CFBC121ED97BCC8ED947
:1019D000085F29152C5FB9A1574A4FDAE7481FF273
:1019E0005EC0A95F1512254A3BE8F948A75F571961
:1019F000E565D2120A4A4AF6EA481FF2A7BE655FB9
:101A0000B1404778CB2A0D66798DC2B44CCD1B13FB
:101A1000AEDCD8113EDA6560B9184F5CCB40F17886
:101A2000340EE066CD5F168626CAF220C94A012E22
:101A30003EDA6760B918615CC9A4B64B15AE074BB6
:101A400071EF3B8634CFBA12DEDA794ACED8065F20
:101A50006916A45F79A2554AC5C8A64861EF4286B7
:101A60006ECAB11FEEDCA665DEDA3160C915805F93
:101A7000D9A14D4A25E5AE48C1EE3A861CBE39F1E2
:101A8000DE312460F948A75F57194C67D2120A4A21
:101A90004A90EA481FF2419308CD5613DEDCA39D1D
:101AA0003ED85F60B916E95CC9A2AE4B153C0F4B3E
:101AB00034468274F6BC1CF56CDD9A8050DD3F988C
:101AC0002586095FA7F250291A4ADACA2A1FCDB51E
:101AD000D9AE5FD27EDA73D66ED8005F89162E5FDC
:101AE00019A24F4A4FE4E7481FF25EC0CCCF1B1348
:101AF0008EDAD8F11ED865609916AF5C47A5BC8216
:101B00009395E5467C5FC58668CD5C12CEDC9B0E66
:101B1000DEDA285FD9180E5FC9A2544A158CA9488D
:101B2000B1EF418694CFB012E7D81FA4F5C6CDED32
:101B3000C915645CD9A1B54B25A9064BC1EEA28796
:101B4000FC5F8412034A194650DD26997FB3697001
:101B5000C0B4FBEC265466663A8DCEB4C871EA4038
:101B6000107805F0544BA1F15487CACD45130EDC13
:101B70009273DED8035FD9168B5FE9A2524A35EE25
:101B8000AB489EEDE71429D1F1B41A4A528CCE111C
:101B9000B65FDD869ACA5C4CD477ECB506675A8C82
:101BA000EC86305FCC40F2782886EC6691F157875E
:101BB00020CD4613FEDC95B5EEDA2260B212C4D316
:101BC000C29EFAD676C407E85EFF58B4D2716C4064
:101BD00092782ED2C6481FF25EC0915F1512CBD606
:101BE000036CD1C4A9FF3C864A5F46407C78AAC0FA
:101BF0006A66BA5FE186F8CA5C4CF94A31FC9B48D8
:101C0000C55F57195967EE12F44A939F4B72ED5F07
:101C1000148692CD5B13EEDC981BFEDA2560F91872
:101C2000355CC9A14C4A15B7B148B1EE39869ECE94
:101C3000B812234A3934FC48368D7DB4955FD112F1
:101C40006CDD9A78F948A75F57195F659512294AA4
:101C500005C2484BA1F16087F8CD51130EDC9E5DA3
:101C60009B48C55FD9DD975F10B2ABEA94424066EE
:101C7000368D7DB4DD5FD1126CDD9A40F948A75FE7
:101C8000571997659512294A051A444BA1F16487A3
:101C900030CD55130EDCA2959B48C55FF086085FDA
:101CA00047A5738461A4954891F143863CCDB21257
:101CB000FEDC81B2EEDA0E5FB612C4D3C69EF6EA3F
:101CC0002CC0C8481FF25EC0145F8212DEDC83CED7
:101CD000CEDA105FE918D65CF9A45F4BEE5024C44D
:101CE0009CEBE512435FDF126CDD9AD08248DC5F2B
:101CF000C918F05CD9A4614B256A5A4BC1F14E87D3
:101D0000E0C846C756DD63B851F7DE1D2816C1CFBF
:101D100056A26DDA8485B1D9F0EE1815A3CEE6A1EE
:101D2000FDD914B321D980EEA81565CE76A18DD941
:101D30008DA491DBF0F03817C7CC86A43DDC703E53
:101D4000C248CA5FD1AC31A3C9A6F678A5DC4A481F
:101D50004485708264CB0A40B17893CF26727C5F51
:101D6000C586DC5FC138D54605FCC66631EF2286E4
:101D700043796E0E8EDEC8580D661FF2C1C0A25F99
:101D8000821226575E9BB4570C7C306579CAAEA58B
:101D900035DD4C07B4DCE2550F8645CF86A25DD910
:101DA000743181D9E0EE511A545FEFF153DE6C3A91
:101DB000F4DCF255E7B446BEAF665491092CD11E4F
:101DC00091F122865402A0404E296B9EA801F5EFA6
:101DD00038DC32CD5D12467884FEB9B401F340841C
:101DE000E39EB9A63FDE84A8BEDAE95F511AE6CBCE
:101DF00006A3BDDBF46721DBA0F0E81753CCF6A304
:101E00002DDB6491B1DB10F0581815CD86A43DDCB4
:101E100085C15E99DE15273C71DD3394E9CC219CA8
:101E200017486B5F696516BEE0126CDD961697C9A0
:101E3000EBDE3405C8DE512782397CC1AEDD0856A1
:101E40003919875FFD127E29B5A9F7481FF25AC0DC
:101E5000D7A355D1234A3956F948A75F57190367C5
:101E600062129A4A4A64EA48B85FDF8662CA174A31
:101E7000F94A31729D48C35F5719BC67FF3F3577F8
:101E80000DAF9767F28AE165717052D1234A398E9E
:101E9000F948A75F5719C86762129A4A4C9CE848EC
:101EA000B65FDD86AACA144AF94A31AA9D48C35FC3
:101EB00057197467FF3F35770D979767F28AD16698
:101EC0003870C23EFB762DEAE264CD5F1686E8B933
:101ED00076FFAD38D83150DD269954B2C173613EDA
:101EE0009A762EE2C6481FF25EC0C273753E074A5C
:101EF0001DF050DD26997486C45FC940EF782DD25D
:101F0000E264CD5F168624BE7700AD2ADAE950DDA3
:101F10002699E486B85F8A12104A938F03701FF2E5
:101F200077BFFE5F8212CA4A532581557ADFC30606
:101F3000BBDFD5927E29B5D7F7481FF20BBEB9A1FA
:101F40004DD12EDD46D18F41E4F20F8643CE46A11E
:101F50006DD994C381D8E0EF681655CFB6A14DD99D
:101F600064F191D9D0EEF815F7CEC6A1DDD9F4FF12
:101F700001D960EE511AB9CC96A34DDB84EF51DA4A
:101F800030F1D486185F7CA685DE9C1E59DC67463E
:101F90000EB3C8BB9C3FB52C6AB701AC068C099F39
:101FA0007154AB1B5153A5476EA9513EA868A0CAF6
:101FB0005C4C054A1BB450DD2699F0862A5F47A584
:101FC000738420C2F248713EB9654AB2D6F46CDD22
:101FD000E2E8C548BD5F10866E5F47A57384CBF00D
:101FE0000966798DC2B42D5FF3127DDA947CA1D994
:101FF00000EE28153BCE41A65A4A50FA34A9813E3C
:10200000571995652F9C8478B5E99748996DE2A496
:1020100063BE6B209168FF82BFBE936DDCA48BD53D
:10202000CD9C66DEB4B761DB60F0A81743CC36A365
:10203000EDDB24A1F1DBD0F01817E5CCA6A35DDB26
:1020400094D241DAE0F12818488E49E12B0063F878
:10205000A2487694517532B82E9CCE2909BBCEA9E0
:10206000AD5F6FA0535561B0FE4AAEF40E4449FD1A
:102070009992637A1394A7CC09F0CBC03D5FAFA9C6
:10208000F77AC6122A6D62A32848913ED965955FFA
:10209000E9FBE8772B7DC467B23EF3B32D72D5948C
:1020A000E9CC1022C2C899FDD98623C1791EF6E871
:1020B000B5BC4F6D33FB09869BC3D91E90E615B2A4
:1020C0004F6DBADF03064C51D2301A4A052DCEA906
:1020D000B85FDF86DACA314C034A19DA50DDCF998E
:1020E0004186C3CD78A4ED4AB06862C840BD88D4AB
:1020F000CCDD629422555AEBB855087A73B5CF5BA4
:10210000C8076DD9949551D920EE2816C3CF56A291
:102110006DDA8483B1D9F0EE1815A5CEE6A1FDD90C
:1021200014B121D980EEA81567CE76A18DD98DBACC
:1021300091DBF0F03817C9CC46A47DDC54AE81DACF
:10214000FD5FD486CBD7C134673DE58B3F5C8263AE
:1021500052790E9ED212D54889997C6E44856FA023
:102160005755A7995D6D4E66E9481FF2E0C0C25F02
:10217000204156396FFCA5C0D85F8C65F451D03032
:10218000A8DE6674D044B07BF286C245101CEAD249
:102190002218D052B0699124085F00B08E56DD003D
:1021A0006E4422821286115F47A5F584F3A2215660
:1021B000361ECFB424BEB5124C5884A4B2460E7D50
:1021C000090513DEB5128FDF73C6A156FD6D46A457
:1021D00050DFD892EA6222DEDAD6A15FCE24EE5337
:1021E000DDB08E5696C19748C85F57197B65251E8E
:1021F000DB669BE5494F254EAA658ABE5E106309E2
:1022000085264F6E17796090099EC212264A649EF9
:1022100091D830EF5816E9CEA6A13DD9548D56DCA1
:102220001FF28B87DCCA61F1E62A15CB51FF09F258
:10223000F11AB2CD29116D07A5AA3E49102D6D1DC9
:102240006CC4C3F1EE2993D37571923E651ECEBE68
:10225000C9A4BA4B8DC0DFA991F1498652CA464242
:1022600066DE0C5377B8998E8979EC6EF905E279C0
:102270005585DF7919528845659EC341973A104FBD
:1022800076BD998E4A760F6EF806680911BD77B84B
:102290009D8E4976196E30068109930FA26A19F353
:1022A0005719CF7941A66CDDE1B350DD525F511A69
:1022B000BECA5922C678E6E7D7AEA33E5719D5481D
:1022C00047A56D7A8D5050DD3D7A511A4CCF491299
:1022D000E66C9E2750DD3C6F511AD4CA0B1366DEA4
:1022E0000601CED89960DA9668BEC9A4E64B0E08FE
:1022F000CCA91FF23099FECBC9A2BB4B156C004B89
:102300002DF9874504C9E801DEDAE109D66A3A52B7
:10231000C9164D5CC670DEDCE41B4EDB6D605917E0
:102320007E5C59A3BB4B95B53F4B21F0A98726CBCB
:10233000A9A2BD4B7316D7B891EFA987ACCF2813CC
:102340005FDF15D03F4B91F1A987CD67D816863A4C
:102350006C6166BD013E2ED6A511C9926CDDB64EEC
:102360005289FB8E9A79EFB9DBF16CDDE57BD7AE54
:10237000A33E5719934A47A56E5A95E9014B19F3A5
:102380004A1B12CD1713DEDCE28B7FA99297DB8C00
:10239000B0AEC9A24F4B93036F5819F3296D6EBEAF
:1023A000C992DEB30526BEA2013EC9062C36C994E9
:1023B00066DE6558AEA991DFC9E73ADDCDC6DEB36A
:1023C000097C56DCE0F1CD36463ECDCAE8FA0DA9CF
:1023D000D4F0960FCA0453E7C2C2E5C210644EDBC4
:1023E0009C5E59176E5E59A3E7499579D64921F04D
:1023F000FD85E2CCFA1176059C45DED8915E091682
:10240000B05E8983DEC14D2CDED82A5FCAB55FAAD3
:10241000C9A4DE490586DF4991F1F9859CCDF81103
:10242000E20697E3D7A991F1C985A2BEC9A4DF4905
:1024300005A0DF4993BEC918B95EDAF1EEDC353F7D
:10244000DCA991F1FA85D2E3CCCEA3FEB5DCDF495D
:1024500031EFFA8541E259A3DF4995C9EF49271ABF
:10246000CB65F2BED9A4E34905FADA49953EC9180D
:10247000C25E0CCE8EDC06777EDAC25E57194C66E1
:1024800085347F39931190581FF2229643CF41A68D
:10249000EEDA9E92D75E324EC918835F47A5405A46
:1024A0008D34BEA1013EC906272BC9943E34754F19
:1024B000DEC8A0D5C908BECBA9FC4E29053CD13445
:1024C00091E1CD3A4B2BCDCE66DE062B56DCE0F10A
:1024D0000D6B52BF2AF16CDDA7D1D871724ECD665B
:1024E00070BE47A56E8146B7FFBE21F02086FECCA8
:1024F0009F12DE298635DFA9E0EF511A33CD96A46D
:102500004A4A1482D66A2A5257195B4C4BD16CDD69
:10251000E10344CBF0EF181610CB86A43DDC711E0E
:102520001866913FAB6528CA7A19DEDA0A2BD17694
:102530003A52C96655BE03926CDDB83381D8E0EFDC
:10254000511A9E5F5EA7FADA9CDEB866013E5B1BFD
:10255000DCCF5BA8449E7B1FBAD8F9FD39864F7A41
:10256000D0349F3E744AA14610692918E45EAF40FA
:1025700049A37593B81C07A62D1668C8C5A270E0BC
:102580006D1EAE48228238B47751B61C3EDC388FBF
:10259000381CF78D3965700BBF5942DA970BD2D8CA
:1025A00023F53124545F58354D7884A4A142F1F1CC
:1025B000D385BACBC640DEDE052AEA49F78D34DF83
:1025C00030BEAF66549169564CDF9DEF5B1C26C14F
:1025D000B9126F6D14FADEDC981BAFDA3A71B9F1FB
:1025E000449E7BABBAD823F4D516F8C9A1B04E4AA5
:1025F00096D5D16691F3D142F0CBB512E0CA0DDC8D
:10260000DFB994DF6F0636BE61208F66098CCBC8B8
:10261000396D82A43B617816773995EB71A6413EFE
:102620006B082ACB86A43DDC7128D1C899816279D8
:102630003ECA8722600993A387589CDFD308F05FC6
:1026400047A55B5B64D491D819F34586CBBE96123F
:102650007BDB0FC6B7BE9F3FDA65CBDDC994C5CC27
:102660008DF4A248983E288675CCC3A647400F8DAE
:10267000CFA9A2E1C9087ECB46A47DDC54EE81DA65
:10268000FD5FC966E1BE47A580519A6D566620BDC3
:10269000C966F3BE03926CDDB891D66A4A4EC9662C
:1026A000C2BE09406CDDB8AFD66A22525AD52FA9F6
:1026B00096A22DDAA42451D819F34586AEDC47A59D
:1026C0009A5C8D56A24834DF6B08C4CA752466DE56
:1026D0008D44E1DBE0F0281737CCB6A36DDCA44CC9
:1026E00091DAF0F14955E9CC84C83C003BC3244859
:1026F0007D5F5965F4BE6ED12C4A866DE848543E24
:1027000099650CCA484D554AE5882FC85CDFD2064A
:102710008ADF19F16CDDAC2B75C8085FC9068FDF45
:10272000CB20EF6616A6DECA9ADF31B4D6DF4BD1D6
:10273000EFDA8E3CC066A979DB9CEAAD5670E129E0
:1027400015A19647EA7C649AF1A8C9406DD994DF37
:1027500051D9F0EF181649CF46A25DD974CD81D971
:10276000E0EE08156CCB46A47DDC54F881DA20F04D
:10277000163CACE9C094E94A80783EC882DF1786EF
:1027800081C808F1AE2993137975095FC9061FDF67
:1027900048A7EFCC051651D9F0EF181683CF46A203
:1027A00066DE443191DBF0F0381755CC46A47DDC71
:1027B000542281DA112E581775E997C81477FFBE95
:1027C0003248213E4965E19E87125FDF3BCC1DA95F
:1027D000613E5719D562BE12BECAF65A15C89ADFB5
:1027E000E306B2BE47A57585B068A94891DFDA0651
:1027F0007251D82EEFCC0574D7C8F98D4306FC9ED4
:10280000D8A26758232AC652A37519781301CAF1B2
:10281000EE294D1D87572C73027B9A7146A16DD905
:1028200094B181D8E0EF681627CFB6A14DD964BF27
:1028300091D9D0EE511A39CD56A42DDC64AE51DBBE
:10284000DE15273CC85FB512BECAF6CA904812F41E
:102850008A6502BE47A575857D58DEC8A2DF4A1B82
:10286000F1DDC994E7CA94F781D8E0EF681661CF2B
:1028700041A666DE74E7A1DB20F16818B3CD96A40B
:102880004A4A3182D21EB0AD2786EABE3BF45E2AA8
:10289000987172D834915175E4CD5AA78ADA9808A4
:1028A0007D7A294E5C1BDACD5AA874DFB13C48DE34
:1028B00034916175A2C835A474E0162D72D8A2F5C2
:1028C0006CB5E2AAD8A77ADC165E5B89328F617597
:1028D00041C845A4EFE081D67EC8358E5175CEDD66
:1028E000B5127ECAA7C637BD221E42860009B66051
:1028F0004EC981F2BEC90F725279EADC66709D98AA
:1029000086C1C048F38D35A0EE493104CDA8969913
:102910005FDF748E5275AB91D9F13C4A3147E106C5
:102920000B5F34DFDB116992E078145A78B4151E1E
:10293000CEB562AECDF16609C1A86F793252D2B57B
:1029400058AEC1F15F0905A77E3739896908D10101
:102950000670BD981B657FBE0F5F36DCA311C99260
:10296000E1799593DCA991E1D12EE86E5901DF2937
:102970000DDAA048F9B748D4F8DFCC476E39099989
:10298000DECA0F5F38DF7911C992E079957DDFA942
:1029900091E1D1321F6B5901E82E0D3416E4400746
:1029A000796528BBD9F1E26416A0DC5EA46565797F
:1029B0003ABBCD2CEDF40F1ED4792152D36534F5FA
:1029C00096A22DDAA45451D810EE3815C4CB46A4E3
:1029D0007DDC544081DA112E163C04E9C5126CDD11
:1029E000BFF544CB2AE0C965565F2670DD98937B1E
:1029F000ED5A9D40DA6592BFE712ADA8E4B250DD12
:102A00007A7107866B0136606CDD3818A648FEB512
:102A100048D492DFD9F15FDF1B8CC6669985E01A36
:102A2000A7CBD394E7CC06C7E04880BDC8D420CA62
:102A3000FA24EA3515D53EABBF5F98E4631147A58C
:102A4000C75C4342311690AD5719F94D47A5A84AC6
:102A500094C151D9F0EF181647CF46A266DE815EC9
:102A60008248B3B808D47BCC55A373F799C3824886
:102A7000BFB908D469CC55A33A4A2D20E1062EF0FF
:102A800065175E5FE96B1D98A21B42DB280C5F3364
:102A90004C5FE56C1D98A20542DBED5FEFE0211174
:102AA00054A37ADB61A4F010D0AD6617B0CC9512B8
:102AB000FEA544FC43DB2DF025861005F6606FDF94
:102AC000A15340DBF5B948D4D9DC59936EDB51CD25
:102AD00056DCE0F0281739CCB6A37DDC544E81DA01
:102AE000FD5F2586D7BE63F1A129FA0B3CAA6F3E94
:102AF00037681C70A7005C7777159167023E28B392
:102B000011BE65A471DFD1944DDE27F4C51818C934
:102B100053A7CADC9F82A348F9B548D40CDC54A75C
:102B20007ADBA2B40EDF6DF1991CD65FBF9B43D355
:102B300059BF9DC7A2F49518A9C9DEA78ADC1CA8B5
:102B4000CADF2DF1DD1CDCC855A3F8E0824CB210C1
:102B500010AD59078DC865A437E0B60B4FDF13F4ED
:102B60007CA81BA856B7E22F0EEE45C32DE847867A
:102B70009C04B6606ECB8376B51310ADDA65EEDDDE
:102B8000B71248A384CACCA9A1E147866504B66000
:102B90006ECB8392B61310AD5907645FAE6B5D9830
:102BA0001841CECA0F5F2FDF5711DDF1EECC83AE97
:102BB000B91010AD5907485FAF6A5D98953FA048BE
:102BC000FAB748D45BBED9945C4A6D92A10621E065
:102BD000D72CCFF851BB77F3073AD4E22C08D16752
:102BE0006FF5CDF2E6F84AB0810629E0281621CF2C
:102BF00056A25DD9746581D9E0EE511A33CD96A401
:102C00004A4A9397715CDF5FCEDF95116AF13A4AC9
:102C1000073E43DB9BF3327CE65FA4695D980BFFC4
:102C20008148A98D6617BCCBA008DECC832CB611D9
:102C300010ADD065B4DD871222DF613ADC662EF07C
:102C4000D31AABA9B7123EA484064ECB0F5F38DF70
:102C5000AF1159935C4A670CA10631E14786BF0565
:102C6000B660DF2905E6A048FFB848D47CDCB7127F
:102C70004AA0843CDECA0F5F34DC8511CBF1DECC88
:102C80008380B41E10AD5907765FA6695D98960DD6
:102C90004ECB0F5F2EDE6911C3F2F02B161EDECA7B
:102CA0000F5F2CDE5B1158936ECB83AABF1010AD63
:102CB0005A07A2DC80683D989D3B81D8E0EF511A0D
:102CC0000FCD96A44A4A9353A05CDF5F5719A74BD8
:102CD00096A22DDA8D40B1DB10F05818C3CD86A432
:102CE0003DDC853393FEEF15D5861C70B5124BA0E5
:102CF00084BE4ECB1FF2A99BE2DC50932C4A86691E
:102D000050DD2C72D1A8D7AAC5F3EF29E9ECF04821
:102D100060BDA8D41ACA98244677531A5FDF1FF201
:102D20006499CA485001264A93BDA05C095F36DC0D
:102D3000CF11C992E17995C7DCA991E14186D30908
:102D4000B66055458A85D164948E5575CEBEC994BA
:102D5000DECA15B35FDFA7F3E1B4D279DEA6E5DE04
:102D60001FE2D7CADF5F4A1B66CA5225E079559B2E
:102D7000CEA90D5F37948941A12057687126A0061E
:102D800091DFDA06E6DFE712ADA8E4C450DDE271B8
:102D900041B35C5F48A76CDDA08DA65F2A4E11860B
:102DA000AECA2026264A9333645D20EE581571CFB3
:102DB00086A27DDA9424A1D900EE511A93CC76A391
:102DC000ADDBE45131DB90F0D81755CCE6A31DDB29
:102DD000544381DB00F04817D7CD56A42DDC644C5A
:102DE00093FEEF15781CE9E8B1A53C08945393F6DF
:102DF000963E2C6607BE96127BDB0F6EB7BE21F0A7
:102E0000C78512CC25115E3798E9D0A5A33E696528
:102E100020BE1DF7C0297333BDDD51420DB36FBE17
:102E2000CE3FEF7525C7F467C14DB4B394B3323FBD
:102E3000864AA1328748243EF394814153A63F40FD
:102E4000275AED42BBB205D46B6E69054F4A79D85B
:102E5000DEC8121ECC6542C8C5A472E0765CDEC82E
:102E6000F98D38F66DAA21D13F990A947B89F58EA8
:102E700051752D9EC740EE296178F317CDAD95169B
:102E8000C47D4001B409CD36A248F6B947D4FEDF6F
:102E900039A6D26CFD2C1ED88F5E45867D05B760A5
:102EA000224A85235C89996DE2A4A0CAAB08A67466
:102EB000C5222049BDF08B453EA155D1DEDA98BC34
:102EC000D66A2A4EC9B96FAB70D1DEDA52CFDF793C
:102ED000AA53D13644CF0212E7740D62DED87D5E6C
:102EE000D2B062CD2511AEDC9DEA3EDA795E0917DB
:102EF000E35D6DD142796D03AEA9A05F56E3E211A7
:102F00009112EADA0D26F7BD990F2886A905F76018
:102F1000FADA0E38D6F091EFB58586CFC03CDEDC0C
:102F2000F121B6170DAD990848CD2111564A65AD6E
:102F30005B89E25F6517349EB8126ECB573C33DB7A
:102F40008EF076866B01766066DDA6576F55378EFC
:102F50007A8A5BAE26E0DE2B05CA494A39F8B965A4
:102F600047703DF195778E804CA93B4D7C6554DDD3
:102F700060944538135BBDA9AF8C466CD370BAF131
:102F80001D77AC636DA94DE17408125F606E9D986A
:102F9000C31273CA3B417C65A0D966940C2AEFB179
:102FA000FCA98B8C0369ED70FAF1B9771DAC711433
:102FB00050AD830C9DD969F59129C13C75CE354141
:102FC0007C65FCD964984C6D84ED7064338E6279B5
:102FD00050CFEC1364090637CED8BB60DBB5D7AE53
:102FE000C9F1304A11763948743E1591314223A611
:102FF0003F407BF2B050106738DA0611E09618CEE9
:103000001290E4CEBAE5CCB500AACAF1E2CC540ED7
:103010003EA9813E780C18CA5817554A7312A1561A
:10302000FD6B46A2C909B5606FCB95A9D1A6B04585
:10303000DC08B0DDE2961ACEA2ABE2CEBCE5360AE1
:10304000BEDB58A36FDB83C0B3CE40E36BA807AAF7
:10305000C9A2354B15C4864BA1F1C788DCCD341409
:103060009B095762D2D899817A76995FC992EFCA43
:103070005A704FDFADF1D718596E0005BEDAA57D45
:103080002ED83260D66D17BE47A5B44DAC4DDED8F4
:103090009564D1A88DAF89A10C4A550BF14897488A
:1030A000DA65ACCA8813544A6DB2A74201F1F886BA
:1030B00050CDE71271090526DA4F99815A799C6E35
:1030C0006005314A1254C2D822F54E45345FAB6BCD
:1030D0005D980552CFC8065FDA085ADD9C12CBDA3C
:1030E0000170D66E885BC91A707147A5BF8361EE07
:1030F0009548FCDF450677CDD8A4FFDC366EA2CA22
:10310000FCE1F606BADF64A21CCC32886EA991EF0E
:10311000138782BE4FA76009A7166D569BF32B7CC1
:10312000CFDFB1967FDCB6B4A6CE00E121867BC8A6
:1031300064A29ADADBA205DF5EEFA51660C9C8F1CA
:10314000A060D84452B9913E3D86CADDC822F84AF3
:103150004E5050DD0C96F206E2DFC4A4FBDC3FDCEF
:10316000F7CA055FC906EE7D7801364ADAFBD3D887
:10317000ADEF9F1C779EB112E1D619F650DD0C968B
:103180001A860FCDD4A47B4A8D1DBF55027A57E411
:103190008F1141A5DF65168BBCA9013EF793214035
:1031A000271FDD678D311F55627A3C654348B8158E
:1031B0006739907C4EDB5A616916585CCB40EE292A
:1031C000CB21CBDC98F3931A29A9D140DEDC8BCB41
:1031D000D66A2A525917DE5A4FD1EF99154E584DDB
:1031E00040D16918EC5A69A2414B07C4CEA9473EA9
:1031F000DE1A75CB73A63F401DD6DEDA1862D1A861
:1032000039AED861EEDC8C03713A31F152890C9EF3
:1032100059A3674D0AF3CDA971EF2A8712CA5B2122
:10322000EB2D18C33ED8BD605719384EC9A2E04BEC
:1032300093A5784F923EC918BC5866A76DFF7DAB29
:1032400080F6201C164499CF86A27DDA94DCA1D9A1
:1032500000EE28159BCEF6A10DD924CBD1D990EE46
:10326000B8153DCE06A19DD9B4F956DC30F05817FB
:103270007FE846A36F6D74E5A1DB20F1681851CD9E
:1032800076A4ADDCE41631DA90F1D81813CDE6A4BB
:103290001DDC540081DA00F148185CEF47A52F804F
:1032A00011A03ED80661B5AC68CDBC14D6DD553E44
:1032B0001548878DC6A86A7D1AF24377D85DAB673B
:1032C000B13EF965335FC8A2DD4A05FFFFBC8881C6
:1032D00052798C9E9434673DE019DED8FE61D91690
:1032E0000E5DD1128664BEEC4EDAFF614918035DB3
:1032F000B2F18784C4F246B921F03588B59E8012B8
:10330000E3A118431BA9948FDD8C72AAC9A24A4C71
:103310000D2106BDF1EF3588E8BEA7205D68694143
:10332000A20642E1690836CC5114DEDA712ED116BC
:1033300091F13588199EC841B73E823ABB120FAD54
:10334000C906DA71DF347F3A116AC348336D7CA451
:10335000D87D8005574A6806A20691DFDA06F65F37
:10336000012CB7544F64DB16A29E3065E362D71878
:10337000D63DA92E62060A5F9A083ADDB41246A726
:1033800081CE4ECB161E6CD6B411B0126FCC850C0C
:103390004FDFB58EFA8A9FAEDCE05DDA740C81D81F
:1033A000E0EF08160BCFD6A2EDDA043A31D870EF71
:1033B00098168DCF66A27DDA9428A1D900EE581513
:1033C000CFE046A17DD99D524489F1EF3F883EBEB2
:1033D000A46F5A980554DE7B7A5229162A5DB9F1FA
:1033E0003FA483ACDEC891C2C918965EC6FDDEDC80
:1033F000FFF156DC91EF3F887701C9A4544C056E6C
:10340000A84A968E59780ECB31A57DDB949F51FF4B
:1034100020F05AA93BCD76A4ADDCE48831DA90F1F6
:10342000D818BDCDE6A41DDC74BAA1DA91EFC18530
:10343000A0CF30119778A5D7CEA99389DCB01ECF45
:10344000BF148279AEB1CEDADF5FC918815F5CD17B
:103450007EDA7B507A7999522916AC5DB9F1E29BFC
:10346000212EB046107D2DE29411D894DECC65FE5D
:10347000A84A013E31E38A115993DEDA7B7ED116E8
:1034800091F13F888ACAAD2A5DDA741AE1D8C0EF9B
:10349000E8161DCF36A2CDDAE40811D850EF781621
:1034A000AFCE46CF6DD9A43746DC0D5F24862EDF24
:1034B000D5A2EECC112656DC51EFA88611B9FAF14F
:1034C00045367723CEA9161E7616F7CF68A48FDC73
:1034D000248ECA5EDA55CDB5C1AECC41EF3D8E1F0C
:1034E000DED8DF60D916295CD9A42C4B057E914B20
:1034F000191EC9163A5CD9A22E4B1568904B91F152
:1035000019878BB9DBF16CDD6C1D56DC4015411958
:10351000F871B9F14C588408BA140DADC9068FDFA3
:1035200066D066DE94B641DAE0F1C916AB58C84100
:10353000C73D05A2D64FA1EFD28B3AC97001DF2952
:1035400015A1CEDA9A64C918C05863D1DF2905DC09
:10355000D94F913FE067C6CDC017DEDC0D5B9EA959
:103560001A3F5965739E65408E297E6AB046107D6C
:103570002CDD8E1158936ECBA5E69E4832FDD99274
:10358000B0C1D91E6F6D11DFC006713EB96580CA2A
:10359000B9132DA805040148D975717892CA1A1279
:1035A0002DDAA43251D819F3781795CC06A3BDDBD8
:1035B000F42321DBA0F0E81717CCF6A32DDB642D54
:1035C000B1DB10F0681809CD96A42B00637A72DE87
:1035D000201441190AE146CF2B08A54AD64F41EFE6
:1035E000D28BDCDD6494E52BA5D8664E1A4E894556
:1035F00070CFC212EEDA11F6CEDA1C62C918F45A94
:10360000C9A2464C1594B74AA1F158898CCD4715EB
:10361000DE2915F3824891F15B898ACD5A15FEDCCB
:103620009925EEDA26625917335A59A3784D95BD7C
:10363000D24B31EFED8606CFEC128EDC92397EDA7A
:103640001D626916AE5D79A2494CB5D84F4D31F176
:103650005989D2CD5F15EEDC9C5DFEDA2962F9183E
:10366000795A59A37B4D95F5424D21F0D687BD9EE1
:10367000E1FF11293FF2F7CE4F3EACB348BE3A3FCF
:10368000A82A29AD1AA9C58C356D78BEB39447CC4C
:10369000D770DB67653EDEB3B3B678F19ACCB01C69
:1036A00034A9578CAD65F0705DF107CE3F28B3D8D3
:1036B0000EEF030C1DD9B1984DCC58BAD3D8ADEF4D
:1036C0005A1C6D5F012CB7544FC809B6151ED1ACFA
:1036D0004979CD2CF3540AE1CF4C1D52954535DF85
:1036E000B5927EC9B6658C489EEFE5161D5FA12C8C
:1036F000575454F2F46EA85BE91A40716FF1E65822
:103700001E1EF456CC7D731AD9A9F5122B4AD08807
:1037100002CE1FF2AABF7D5F3512A9CEE198E44820
:103720009985C082A4CBD1406CDDE611C548BD5F50
:103730001086845F47A524822038F248E55FB616DC
:103740003DCFC4A2FADA93D30070ED5F1486BA5F5E
:10375000C994EFCC27D6EDCAE65FD616C0CF58A8DD
:103760005FDF12F0C2DA035F7A074ADCA69256CE18
:103770005870B3DA0DF11E8615CF35A26FE0F04F09
:103780002F4C094EC96516BE47A5BD83208CF24853
:10379000055FA906E5DFCB92F1CA930F98701FF27F
:1037A00077BF7E5F82125D380691C14E454EC9BD1E
:1037B000215B6D01ED3015575F899246F20604DFFB
:1037C000C5A47DA86725AEA97F6CC8A36250F62F5B
:1037D00087CABF52711650AD8308F3DDCDF1EE29D3
:1037E0000DEFC757BCDF0506B1C8F59409CCD3E18E
:1037F0000157278E5275AF91A4925CCA66CDAF4C2B
:103800006252D26C96BE47A5455D059AA24B1FF247
:10381000ACAF02CCCE17DEDA0D1FCED89A644A1CAC
:10382000B0CDC017DEDC0D2172DF20144119F0E1AC
:1038300046CF2B0864A491D830EF4815D3CE96A17B
:103840002DD944D3F1D9B0EED81535CE26A1BDD9A6
:10385000D4C161D940EE511AD8CFCE17E079EEAB82
:10386000DED89964D916EF5849A89739068DCEA9A4
:10387000A1F1D28BF4CDC11766DE079BDEDA986426
:10388000D36513BED9A4E74F051AD64F91EF6B87C6
:1038900000CF6A13EEDC8B94DEDA16615719DC5C1C
:1038A00047A5B14A8D3081DB00F04817A3CD56A45F
:1038B0002DDC6420DED89964D9163358C841EF4E08
:1038C0008E311F89E1EEA886BFBEAE3FD1297CE1D3
:1038D0009EA9E13E4965C6BE62D1E66CB62DA648FA
:1038E000F7B945D464DFC1343F3D83EABC170EAD60
:1038F000A90683DFB712479B82B62FCA71E14786BC
:10390000E306B560CFCCE584D66E885BC91A9671A4
:1039100047A5BF8361149548085FC9088DDDEB9406
:1039200011CC947C410633F4CD65BABEA11F576714
:10393000051E535CA150D26CAABE47A5455D93AB52
:103940002B4B21F0D08BC6CFC117EEDA0E4B5FDECA
:10395000A1F1D28BD4CDC1173DDA54CA41D820EFA2
:1039600048158DCE96A166DEB4FB61DB60F0A8172A
:103970001FCC36A3EDDB24E5F1DBD0F01817A1CC8A
:10398000A6A35DDB941641DAE0F1281841E997C857
:1039900085E09425A6DDEF1D584357E1C9A2A74C49
:1039A00009914FBD243E4A45B8BE49F57E77B6839E
:1039B000DEA6598CD172EE700840AE297FBCBC1ACD
:1039C0000EAD6906E67D4005060967E4B138F2AE42
:1039D00013865A51D0308448A4197ED829616DBB12
:1039E00030AB26C856DD7507B046107D2DE31211A9
:1039F00069928FCA81F4BE1B0DAD7A08DCDD26D03A
:103A0000DECA1682D214A69EDA088ADDC9A2764CD6
:103A1000144EDEDA29616D45E8BE961206A74150C4
:103A200072D83594097949E9B1A54C588432BA1451
:103A30000DAD690605DFB5123E9B81746FCA31E199
:103A4000B844C2DFD892EAA61A09CFCA91E1D516C6
:103A5000DF01C5A463098156BE1B0DAD9A071EDCAC
:103A60005D41663DE6A5A448FF6D48A48C0CB56099
:103A7000BECAF6F276A4719DBB8C73AA1CD1DF7806
:103A800009D1CEA90D5F31E4731149925E6C8E7B32
:103A900015899BBDE4D44A5FC5A1F76D0D91C7554B
:103AA000F14C3C652A50D62F324A323BE2D922F5FE
:103AB000F9741948F1FE194FDE48D66E885BC91AB1
:103AC000587169408E29C5270EA91FF2C1C0A55F94
:103AD0003512134A0DF229B491F3E1B44D5F692C0C
:103AE0008F52C9C469B451F39DB4E4CA314C3A4A07
:103AF00050F09647EA7C33A303404FF153DD6C6BE3
:103B000089DDD8F2531AD7A9BD122FCB458F528920
:103B1000E55F5A1B68CD27A465097F1AB046107D62
:103B200029D7DE1118939ECBA476487919528D546B
:103B3000B0CFCE17DF799EC350DDE5782F47BC6E3E
:103B400050056CDDD859BF8B91EFF387CE6E4005E1
:103B5000B409E5C2B64A81EF3288E2B32950D950A0
:103B60009E90DCA4A43E5719985B29A2354CF5FE23
:103B7000864A9985C082F6CBD1407EDA117F6D6E80
:103B8000385B791AC7711A406CDDFDB0F548CD5F1E
:103B90003F65E7CB2EA6B5DECC0CA4DCE255CD6CA0
:103BA00031BEF3126CDD75A53ED8FB61B916455DDB
:103BB000A1FEBE8803B247B89A4BDC65B2CAB916FB
:103BC000BEDA63C02ED8F061D1ACBDA3C9A6F67829
:103BD000A540D34B44857082E8CB0A40B178934B23
:103BE0002672BC5F058600BE3CA6C5DEDC7819DC0B
:103BF000FBF31A7C79B6D8F1184A936FAE4B71EF8C
:103C00006D8772CF6C13DE2915E950DD7098691647
:103C1000345A79A2834DC586784D61EF708910CAF8
:103C20005C4CDBCC13A6C1CAAA8272B11A7021D334
:103C3000007540172B48FF6A48A1AF5F4AF18058D2
:103C4000B85E54DCF255830861DDB0124C568452E4
:103C5000B31E0DADA90A27DB2826CF4E6EAC3B481C
:103C6000DD6A26A1A852942DE529188B9647EA7C97
:103C7000D1AC05A3C9A6F67893ED3F73FEDFA70686
:103C8000CFDF4A3E7C78AAA86A66BA5FE18680CA1E
:103C90005C4C344AB20463D85EEFA51692CA174A48
:103CA000F94ACB8C0D66798DC2B45C5F0994AFCCB8
:103CB000E7322DCA985F4CDDA4111140A778079018
:103CC000CD66B68DFDB47A5F84126CDDB3F78248A1
:103CD000DC5F418645DDC994DEDACED8DEB415203E
:103CE000320518DEA3295951A6036DA9F36C3CA334
:103CF000275F5CA7CBD9016748DE065F29E1021187
:103D0000B59449CC073557BD9C1F3A65FE4B41051C
:103D1000B1099582F44B228E5275549E60F28E2921
:103D200027BFAE48B4FC39929AC0B91E6F6D717747
:103D3000A00697DFE006EA5FF412E670FCC0DEDC66
:103D4000A98D3E86A306B46080EEB86C79B441F3C9
:103D50008CB4017147A5D68461589548F73EFE1A88
:103D6000C7CBDEA6E5DE6FF28FBE71EFC98B1ECF2B
:103D7000C8176CDD6D4DE2489E42DC6572CAD121E8
:103D80001A4A4C8250DD0163340676DF5994234A87
:103D90000D9EC7560D5F36E06411C56DFA98619EA1
:103DA00073D84DEF2086B3C8C4A2FADA9B3A765294
:103DB0004A697A0894DD4ED1534A73B4A156FEB9CC
:103DC00045D4D3DC5993334A2FC6E556B1B005D458
:103DD000FDCF75A26FE06D3A7E764F655279FE9FFA
:103DE000C9A2A74C0AE459112EADCDB5B5AEB1129A
:103DF0004AA284BCDEC8AA85D0826ACBCB20F168F7
:103E00001292C2DAE95FDD1B24CFDDA8234A0D0040
:103E1000C756328E5275829EB5123E9B81523ED855
:103E2000F160C906B5DF39F16CDD6D13E2489644E7
:103E3000DC653CCAD12147C97FB9B4510C662F70EB
:103E4000B3BEA71F5D675D46C9DF3DEF7965CCC195
:103E5000F912E1E8F558CCD6816B5AA99B5F47A5CA
:103E60004E4E05F2944BF43E39658245B81A354AF8
:103E70009AE753D82DEF5F1C76704BD173DE8CEA36
:103E800054DDF3554A9A975B400528097A8CB71997
:103E90000DADC9061C7D50016EDE860E4106716CAB
:103EA000BAA3875F0D1DB365C94ADA67543EDDB317
:103EB0003452DC2D524AE5362FC89985C0823ECB5C
:103EC000D1406CDDE6FF35488D5F018644793E0EBA
:103ED000DEDE1DFC50DD7298360684DF06926176C8
:103EE000A3CE7B66458DF286705F47A5738420EE76
:103EF000F248D85FFF86F8CA174A6CDDB3C782481C
:103F0000DC5FE586F05FD894DECC77EB715F1A5208
:103F1000D045E05FAF615A980598CFC83975828C5B
:103F200034AA9D12BF097726BE190DADC906BFDFA1
:103F3000CB28F15091C52A89055FDA08BCDD39D15B
:103F400067CA9FC254502C6753D95611BC12479967
:103F5000811E7EC80D5F29D7A411C992EFCAA77C24
:103F60006FB9354D7A654E45701C274A87ADD21919
:103F7000AFAD6E8630521C2D504A6B2BA20691DEDF
:103F8000DA05EE5FA7353545651DA065035F29D5C8
:103F90006C11C992EFCA0D8EC740AD5F8DACA9A35D
:103FA00009A6B2784CA4E8481FF2C1C084B07AF1E7
:103FB0009E29D55350DDF199FD86D8513A30264AD5
:103FC0009355AE4C065F2FE03411C992E66C063F64
:103FD000CC483DBA85D43FDFB392486280D4B41D4B
:103FE0000DADCE0672DF90126FDF2178D0DA291E78
:103FF0006A6519DFB5927ECC27F813126DAD3206D3
:10400000FADFA32A59526F53A206EB5F761632CF1E
:1040100058A8E3CA1B9476464A7D5A1B20CD67A454
:1040200049CA81A2DEC8B65F8D947F41C134973AF8
:104030007F30BD110DAD23869505F5607ECAB6BEF5
:10404000D3D8ADEF5A1C6E45701C705F984B02BD03
:1040500057BAA5D48E5FC4A2FADA96CC386D88829E
:10406000B19F1B5466D17F5EB66C67B841F36A1A84
:104070004F110F6DBA987F763EC982DE6C458CBEBB
:1040800066274F397F84485D2862A5796C0EB5603C
:10409000A1A1E1DC7EC842DF238617CFD5A26FE065
:1040A0008E61BD110DAD8FD5F41169928FCA7FAEAF
:1040B000DEC8A2DF71A08F554CD1C46DFC995C891C
:1040C000404D886C315FA7205D680E4AC4C8F96D09
:1040D00042A43F09B560274ABC265C89913ED96558
:1040E00073DDCB94CFCBE5659B48996DE2A447DFA8
:1040F000F392E85820EAD31EADAD57197B586AA554
:10410000DEDAE402765F1952DC528ACFAF14EEDABF
:104110006C12E6A4919DE48CC9AEA600E67C23183F
:1041200072B99A9ADA8A02AEABF1610965CD5F89FC
:10413000F23EC9167E5FA128AF3965A814481085E4
:104140003082B2CBA5635B9805C850DD426F59172A
:10415000A65D47A542629DCE5C89913E4B45DECF70
:10416000E0136CDDCD7779DF20144119B2E146CF41
:104170002B0864E291D830EF581685CEA6A13DD920
:104180005411E1D9C0EEE81507CE36A1CDD9E41F10
:1041900011D950EE78159ECB66A39DDBD40F01DBC1
:1041A00080F0C8172BCCD6A30DDB443991DBF0F09F
:1041B00038174DCC46A47DDC542A81DA112E49559E
:1041C0000DE997C8FC2A4EE9CCA9EA8C756C6C7095
:1041D00068F11077C23FDD67433EDCB391B92D3FF4
:1041E000A129F9CD09A9568C9C65BF70A7355D6DD5
:1041F000EE107867428A7365C8BEABADDE4A68636D
:104200004E4403FA5992177A45697C985B0C33D86F
:104210008DEF11863DDD73946CDDDB1FA84852EFF6
:104220009A164D5F1594A9CC4D2850DDD2609406A6
:104230006CDF012CB7545A36D3D8ADEF9194674157
:104240001594A9CC4F4450DD2197720676DFF01209
:104250006CDD3068AA4872F1988611DF1592364AF3
:104260009EF702DA5FF1611CBB5F54A37BDBC26E79
:10427000AC48913ED965AA5FC8A4EFDC26EEEFDA20
:10428000405F51196542B82DA72AD56BFA47C67C05
:104290009B657748B81567393556D7AEA33E571991
:1042A000474AC9A25A4B93333D6320EE5815A1CE1D
:1042B00046A13DDA542441D820EF481553CE96A1AB
:1042C0002DD94453F1D9B0EED815B5CE26A1BDD91C
:1042D000D44161D940EE511AD7CD56A42DDC644C9F
:1042E0007ED85A6111B436BE6D41973D51E2835676
:1042F000D1B025D4ADDD0194C209A7CBD7BD0F5FE6
:1043000029E1FE11C8F1DECC510683560F5F36E07D
:10431000EC1118949ECC4B4B82068AE1B1084F9E5B
:1043200069109B0913245E46227D2786BFBEE320C9
:1043300019681FA6BFBEB16DFAA49709F560294A96
:1043400085D1944B131ED194D14143A5404096D9B9
:10435000C2DA9FF14786B602B5606ECB14B2C1AE29
:1043600024F4E518EACD5BA87F48B0ABA648F4B6C4
:1043700045D423DD09942A5862669246EE7D12E404
:104380005C11F312E670FC7ADEDCA98D5719EF643C
:104390009512294A0D16C7CABBE104088E9EB712B2
:1043A0003EA581EC4ECB0F5F37945541EAF12A5878
:1043B00062AEF4DCF25535944541A4685A98963DB6
:1043C0004ECBF0EF1816D9CF46A266DE745FA1DBA4
:1043D00020F168181BCD96A46678953B2648FF6AA5
:1043E00048A1155FAB6F5B98E5682FC8085F2CDDAF
:1043F0000C113894BECC6DF69246EE7D1594234197
:1044000080703A980D2229B491F3E1B402CA284B86
:104410003A4A5012D6CAAAE1F308A1DD81128129D5
:104420000D2EC7563BF32A7CA653D62EEBA0216057
:1044300050DD46652816F9CF56A26DDA84ADB1D9A4
:1044400019F358185BCD86A43DDCA9AB6EA9397968
:104450007A8E38B139F16009EB5629563BF32B7C43
:10446000E8793E0EDEDE1D4850DD7298D486B671C6
:104470008040FC4A0B5ACF66B48DFBB4C05F8412F7
:104480007E2CB76D11AF6A4057199F659512294A66
:104490000502724DA1F1768938CD67150EDCB49B0B
:1044A000C048918DDAB40571FB401A4A52AC77A529
:1044B00049418F65EABC47A5738461BA954891F17B
:1044C000718952CD6015FEDCAFCDEEDA3C62E78635
:1044D0005071D840017837F8E248DE5F766FEAB075
:1044E00007FCAE2C93714B72ED5F14866CCD6D158D
:1044F000EEDCAAF7FEDA3762F918DD5A96A22DDA59
:10450000A49051D819F3981757CC26A3DDDB149D3E
:10451000C1DBC0F00817D9CC96A34DDB848F51DAEC
:1045200030F11818FBCD84C83C00AEBC51FF09F235
:1045300027443DE084D03C4A96AFC7A90E5F5A1786
:10454000DACBA008EC4A8E1841067E5F2A65BEBE13
:104550003E38C546F5C01A6E66858FA00B55B63538
:1045600058DD7347BDDDAA85D082FACB6B389170D8
:10457000AD6A67427F75C88C61AA9F124ADB8ABF09
:10458000105E70655A79505FB5A3EC60248A47BD10
:10459000E95F3517919E67289D50966F86480DF00C
:1045A0007A1BAD01566066DD46B58F55F58E3A8AA9
:1045B000B9A97196B9CA1E32D4C864FD69B2AF7A7E
:1045C000C0B09E7696E17A523DE1720683DF60B01C
:1045D000EE7696F71BD6618B5AA94F45D494A6E880
:1045E00005CC4F6D34FD79B2F97ACA2CECCC060DAE
:1045F000F667953E01B368BFC03FF2291ED33EA9BE
:10460000813E3E8614DC9D127ADB800AB01A0FAD23
:104610003D15E95FA2645C9839887EA9413E8965B1
:1046200070BE463E6F708CDA4EDC7782C0A94E4475
:10463000381B2977621199B5E1F28DA9697A0529AC
:10464000BB51296CF116D95F6082895F48A85A4A2C
:10465000735EA156F96D42A4BC51BC30DF2915BF71
:10466000D246AE7D31949F41D99207E815404F6DF7
:1046700030725D79F5BE48D1ED381DE4DE642282EA
:104680007194445F9E0D204A861EA248FF6D48A487
:104690007851B03042587A88DFA9A13ED5940341C1
:1046A000A12057680524F6D6B18B5AA9B7485D05F5
:1046B000DF298673D1A6B9FDC9B2AB7A7120ADA846
:1046C000E48E1D796263527574919C128BDCE2CE8C
:1046D000AA4842F19886F47D5801916C0E29DFAB0F
:1046E000A53EAB7195BE0AF1AE29937F5F759F3FE2
:1046F000DD6597B238F1A129D51950DD129A4F45E1
:104700006F013660C179F60257B98C2D721B01E832
:10471000B1A53C0894AB93F6F0EF181603CF46A270
:104720005DD974B381D9E0EE081585CED6A1EDD957
:1047300004A131D970EE981530CB86A43DDC703ED3
:1047400084483DEF2BB4B979AE0E4EDE975B1ABDAF
:1047500042F53794AB41A1205768A5DA6FC81C1EFB
:10476000291A92CBA7205D686D66A75631DF7A06BD
:1047700040CB68A69D98BEF476CA22F475166FC920
:10478000AB405D706C78AEDC23748D79BDC9A72019
:104790005D686D9CA75631DF7A06919EA9A64EDE14
:1047A00073AEA156F96D42A488DF78928EDEA63AE8
:1047B00061064CE17308A4C865A270E06792A16E1F
:1047C000F85B391AD6480D058FE073C4A156F96D10
:1047D00042A452DFD8926909654CAEDCFF6D48A453
:1047E0000851B030DECA1666CEDC92F3E8D473DD31
:1047F000C5943DDA546456DC91EFD08B747DF80596
:10480000E2290590D94F1FF29C8604CA2213E6378D
:1048100018F150DD2196CD7489BED9A4E74F058CDF
:10482000D64F91EF1886AB21C9A42D4A8DB81666D4
:10483000988E517572BEC9A2A74DEFDA50DD44665D
:10484000511A8DCD96A41E2955A9A048F2CE39F54E
:10485000BB04B760DECA05C4174D764557197C56B0
:10486000C788E67F7E914EDBE85F5917BA5FC9A221
:10487000A74DF0951EA11FF27C8DF0BED9F16CDD25
:1048800095B9DED85A62B46BCBBE47A59151051ECF
:10489000174D7C3F916698CA7A19DE299309496DB4
:1048A000923E52452EBED9F16CDD95937FDFD594B3
:1048B0001A8AEBA8C9F13DDA542856DCE0F1281831
:1048C0000DE997C88AE09471A6DDEF1D584303E116
:1048D000C9A2A74DE831F0485ABDA8D4FABE79F173
:1048E0006CDD84E4D66A224F8806CABEC196EE29E2
:1048F00007DACD62ABE1D208C1DB69F1E8CE151F62
:10490000DC62A489E5088DDD72967E291188CEA926
:104910009389DCB08ADDC4942C4A868D33AC853E05
:10492000976676BE47A5FB6C06C95F89913E751BED
:104930003FE8B1A53C08948993F6F0EF181636CB02
:1049400086A43DDC93D1006D998152790E9EC9A257
:10495000284B0D70FFBDFE433D65FDBBFDF11F2ED5
:1049600059811DA992EFDA1645CF74A2E06418644C
:10497000CBDC98F3D218EFCD0861FF40AFBDDED895
:104980006E62D916DA5A69A2B54DB51A064D9379F9
:10499000DC9002CD1B15DEDCD69DDED87062D91608
:1049A000C05A69A2B74DB536044D9379DC903ECD1F
:1049B0001D15DEDCD8B1DED87262D916DE5A69A2C6
:1049C000B94DB552024D9379DC905ACD1F15DEDCFE
:1049D000DAD581D8E0EF511A58CF0015DEDCCDDBF7
:1049E00032A8513F5719D556C8F166DE957F144D50
:1049F00021F09289E4CC0115DEDA4CF93ED8D96079
:104A00005719817CC9A2284B939D7F6B1FF26AA91D
:104A1000987D70016CDD7133D66A2A4ECA659ECDD1
:104A20000315052E39C5BFA5033ECF652DCE44A382
:104A3000DF9966C456DCE0F12818F7E997C88AE0E8
:104A400094F7A6DDEF1D584385E1C9A2A64DF0AC51
:104A5000F0485ABDA8D470BE79F16CDD845AD66A8C
:104A60009A4F880644BEC196EE290740CD62743E37
:104A7000DE1AF5CB23A63F401FFAD7CA4AE3696581
:104A80000ADBD9F1E07418AC2DA9A6F3D01AF4CB47
:104A9000A808FACC101665CC313ED50A0CBECB3C2A
:104AA000F1746843CBDC98F3331A4BA9D794EBCC61
:104AB00053B05FDF7E43BD65F9BC1DF16CDD229C08
:104AC000DFA9121EC965EAC846C756DD637251F7F1
:104AD000DE1D28161BCF41A6EDDB2449F1DBD0F00B
:104AE00018173DCCA6A35DDB947A41DAE0F12818D3
:104AF000FECA5236E66C8E03BD8891EFD08B7A6E7B
:104B00004001FD0A0594D64FA1EFD28B2DBECD50AA
:104B1000F0508EE3D88991EFFE878ACFFF135EE0D5
:104B2000B6D5DED8C860D916905C49A8CF39C2CABC
:104B30009D67453E1CB373B5CD3FA02919135FA9EE
:104B4000213E9C65A170B83D680905DAE74BA1EFED
:104B5000038752C92808E02905CA0A486C1E89B48F
:104B6000210E9F122BDA62F63348055FCA16FFCF7B
:104B7000061226645E7E89B6141E191ABDCB966095
:104B8000264A3C8250DDBC99E2AC0DA3D9A65A4A14
:104B9000739EA156F4B844D4445FE320196830CB27
:104BA000E30631DF7A062BCFD5A26FE0ADB66742C0
:104BB000485D4C4584CB68A69D98B1AC634E355397
:104BC0001186C3C8FE126CDD30F2C76E985BD91A2D
:104BD0002C5FA7205D68688DA506ED5FF3946541A5
:104BE000E2651B98A5646FC89EEFE516FDC9612CB0
:104BF0009754BC0C5D8941F36A1AC51165289B5016
:104C0000A1F51EDA655F4F45070156606279960A85
:104C100057B9B62DD565F6BDBDF13D4AA28FD4DC9E
:104C2000FA558916795A19A2BC4DEB0C09B471F3E7
:104C3000BFB4B2CF7915EEDAB63DFED84362F916AD
:104C4000735ACD20F3682B58E95691F17989DECD5E
:104C50007815FEDCB751EEDA44628916035A19A2C0
:104C6000BE4DEB4409B471F3BFB4EACF7D15EEDA63
:104C7000BA75FED84762F9164F5ACD20F3682B60FB
:104C8000E95691F17D8916CD7C15FEDCBB89EEDA03
:104C900048628916F55A19A2C04DEBBC09B471F3EC
:104CA000BFB422CF7115EEDABEADFED84B62F91655
:104CB0008B5ACD20F3682BA8E95691F181892ECD2E
:104CC0007015FEDCBFC1EEDA4C62C9164458D9A299
:104CD000E74F06E3CF4C1A4EF445DACF1D123E776C
:104CE00084C53948DD6A26A12452942D544A65B200
:104CF000A50671DFBA0674DFDA926F299BEB494F84
:104D00002964628B08AA59F1454A51048356D26D31
:104D10001AA2DE5194302BA260567AA6423E8965D3
:104D200070BE47A53E84BEA476CA075F36DED511A5
:104D300089912FC9A121434D4D536B060FDF7E1082
:104D400081097C42B046107D34D9B7118F12E058EA
:104D5000184E3CA9813E5719F3653894BECC6C5E61
:104D60009246EE7D0ED9BB118B2B31531B6C1A6E04
:104D7000485B891A207129F1CE33149BCEA91FF20A
:104D800007C0BBDD6194A80987B957B9581E5AA856
:104D900099AE0DD1BEDAB5932ED84262C916AC5A7F
:104DA000D9A2914D494A9267D23E25B34D72B83D82
:104DB000054A1BB250DDF19979180C5C69A4134BBC
:104DC0009553E24B21F00487A8CF7D15CEDABACBFC
:104DD000DED84762D916E15AEE12F44A9349BE7200
:104DE00041F10187C4CDFE136EDB43E94EDBCE609B
:104DF000A916CA5A39A2974D0568644DA1EF848956
:104E0000A75FDF126CDD653C7E19439E7918B45CA8
:104E100069A4174B95879E4B21F0088795B9DBF164
:104E20006CDD6C3750DDA1665719256F59A3E54F2E
:104E300005A0D64FA1EFD28B39C9D9A4E74F05AC55
:104E4000D64F0E4338B3B2BEB63F233457ADF5AD9F
:104E5000DB8CED658E7059F116371075EDA9AC8CB1
:104E6000EAB1D3720792BDCA7C68DEC8A2DF7106C0
:104E700049DFCB2CF154C6620F4CB24EE586C75FBA
:104E8000C138D5460510C666AB5F8965DCBE47A54F
:104E9000D6842A92CA481FF229C04C5F58A79ADCD0
:104EA000B3325A89E75F5A1B34CDC7A47DA8674F38
:104EB000AEA9FF6C48A394C8871F3D67988DCFBFEC
:104EC000F0EF1816DBCF46A25DD9745B81D9E0EE16
:104ED00008157DCED6A1EDD98D4C11DB70F0B81739
:104EE0009FCCC6A3FDDB3475E1DBE0F0281701CCD5
:104EF000B6A36DDCA46691DAF0F1163C22E92BA88A
:104F00006DFF7D9780F6201C164404CA22136CDDC9
:104F1000D810926DEE8243655770183D6CDDE33B0F
:104F2000D66A1A52AB454EB58F27C9295B2B56BDA1
:104F30006D1EC66AB3703DF1F57766DE3067F53EEB
:104F4000C7B3BC5F7EA7BC4A8DDDFF55C27A69B48A
:104F500063BE48D17E78595613D86EEF96868D5F22
:104F600004A4BBDCC264E6A2DC740465B75818056F
:104F70006ECB96F14CCB24E01E8637CD15A47E294E
:104F800073A5A16DE65FD61615CF1412184AED94DD
:104F90002742DC5FC084959ED9A6DFDE24D2DB7871
:104FA000A2637175A671467084791D5F4889778503
:104FB000A082D2CB3F40DECA1638FCC8C4DFCD94F5
:104FC0005541EF3015680544CFCAB3E1FC08CEBEA9
:104FD0004DD1C5344BFB35A9E78C7AD5E8C87A3476
:104FE00067393D2C56DDF27A3AA12C5FFB126CDD5D
:104FF0001CCA5EDE32525719A45F47A55A780713C0
:10500000CFA91FF274BD0ECA882D2F65F5EA995FEE
:10501000883F208B1CAACBE03F5D761F57BD521EF8
:10502000B086CC7AB635CDCAFDACD7CCABE3F08632
:10503000A65F47A53E840E36C44821F1A1893ECD26
:105040001E156EDC47475EDAD260B40A30DBC496C8
:10505000FCCE2C52C8481FF229C0D35FD3126EDC9D
:10506000DF655EDA6A625918AC5C49A4214BF4EA48
:1050700026C09AE7E30ED15FDF126CDD6546D748A4
:10508000AB5F5918D85A49A4B94D9518984B11F1EE
:105090000E871BB9DBF16CDD6C8D50DD7D835719FC
:1050A000305647A56D7AE73151FF09F22744A1E058
:1050B00084D03DDA542441D820EF481553CE96A130
:1050C0002DD94453F1D9B0EED815B5CE26A1BDD90E
:1050D000D44156DC0D5FC906075FE7681D98B14EE5
:1050E000C666B0BDCB9CA6AA9612065836F04CDF19
:1050F0009DEF5B1C64DD41A6EECC051B56DC30F158
:105100001818DDCDA5126CDDEF214666DF5F57195B
:105110007A7671407E294E16DF46A27B2816D1CFC3
:1051200056A266DE74B7A1DB20F16818E3CD96A421
:105130005E19528480FE9D5FC486309E8112A7CC8A
:10514000EFC250DD7B864086C9CD3612C8CACECEAE
:10515000D0649779CD9CC6AD46A16DD964CC91D869
:1051600030EF58169BCEA6A166DE816AB01E10AD48
:10517000690655A347D13A4A2776EF5423F4B51868
:1051800092C966707ECC8186B31E10ADC9060851E7
:10519000C99466DE940641DAE0F12818705F46F79C
:1051A00072294DA232661FF2FEADC7713E38C54668
:1051B000FF2496481FF2FEAD67CF86A27DDA942EBB
:1051C00056DCE0F0281739CC46A47DDC545E81DA49
:1051D00020F0163C0AE9C51254774BF58967191E71
:1051E0003F8683CF2612264ACE6A50DDC6869206B7
:1051F0007C73C62AE260250451D9F0EF1816E1CF7E
:1052000046A25DD9649591D919F3581813CDC9A454
:10521000554E6D3CBF19F58E9979EABEA7205D68A1
:105220006E7BA00631DF7A0668BE19F16209A5CF50
:105230006CA5523E9965B4BEC9A41E49E5DD27A9F7
:105240009E41D9654ACAF74CE74A1F4A5F19219E19
:1052500069C5621E7FA685DE9CCC59DCCC85ECB48A
:10526000F271C840DEDC4A675EDAD55EC916AF5E11
:10527000C17ADEDC467541D820EF511AFCCFB11659
:10528000EEDA7E865FDFA1F1428A0ACDB116DEDA60
:105290005490DE2B91F1188690CB56A36DDB9429A8
:1052A00051DB2282781899CD06A4BDDCF43E21DAC8
:1052B000A0F1E8181BCDF6A44DDC8428CED8D75E2B
:1052C000C916B75BC670EDC0A558284C937592758A
:1052D00030CF3C164E296E8FA406A1E1C918AB5BF6
:1052E0004BD16CDDC3CCA1D800EF081643CFD6A2BA
:1052F000EDDA046231D870EF9816C5CF66A26DD989
:1053000094BF51D930EE611AC7CD96A46DDB52B867
:1053100080FEF1EFBF8AE6BEA0695898059C7ED852
:105320008763D916515B6028B73915BA284CB0BDD0
:10533000D918445BD9A2D44E244ECEDA87634D45AA
:10534000C9DD47A59C720EC651D9F0EF181646CBA1
:10535000C9A2D34E15C4284C9A79D8FC54CBC9A203
:10536000D44E6C84ABA9F96D3AA2EADF41A6EEDA1D
:10537000F9747ED88463DBA0E729D6481F3C65EE2C
:105380002A4C013E36D57D11C994DEDAF988D11652
:1053900091F1BD8A14CF3D16EDC005082A4C91EF5E
:1053A0000A85223CC9A41F498D3C41DB20F0583BB3
:1053B000BFCC5835EDDC2424B1DA10F1D916CA5B24
:1053C000C9A2D14E1DD2CFB9F1EFBC8A3CBEA461B7
:1053D00059980552DEDAD75EC916A95BC670DEDCC5
:1053E000F8E4DED88463D8FC68CD3A16EEDAF8EA41
:1053F000DED88563E19CDFAAC9A21F491480DEDAEA
:10540000D25E4816EBCFD6A2EDDA949B51F720EE90
:1054100068150ACB47A506720D3A07B9F1EFBF8AA6
:10542000D0BEA069589805A6D07A2A4E5719AA77F7
:10543000B8E06CDDC31C56DC10F0581823CD86A4F0
:105440003DDC7142D0AA1FF200AEC3DF47A5157242
:105450001350501E30AD4186D8DF47A515727D5ED2
:10546000CEC89ADFD29468CAFE3A5D6D8CADA04872
:10547000006B3AA2F6DF47A5157278EFA64891DFD8
:10548000419B2AAD84683D980D0850DDC8872816D9
:105490005FCF56A26DDA840756DCE0F12818F6716A
:1054A000CAF5DEDCF5A14EDB0262096C78BE53A3BF
:1054B0006EDB77B790481FF2FEAD745F47A57A7335
:1054C000645091D819F3981797CC26A3DDDB145DAF
:1054D000C1DBC0F0081719CC96A34DDB844F51DA1D
:1054E00030F118183BCD5140E179951B4ED80D6035
:1054F000CB6A72CD39156EDB76FD4EDB80625917B3
:10550000F25AC6F7F229E62850DDC686D83BF6CA1D
:10551000D9A15A4B9E0077B99A45DB657D7147A5A5
:10552000C95F4EC48CA9643E2EB3DB72A51F5B67B6
:10553000EBD19867E28A1593E54033F1057736138E
:10554000F247CE7C36652870383DCA570253AEA864
:10555000608C9AB11850142F6129EECAD1AFA53EC4
:105560005719D776BE12BFDA0468D1AFA53E5719D6
:10557000C576BF12BFDAF476D1AFA53E5719CB7608
:10558000BC12BFDAE484D1AFA53E57193976BA12FE
:10559000BFDAC492D1AFA53E57192F76BB12BFDA3E
:1055A000B4A0D1AFA53E57191D7648610F3F1449ED
:1055B000CAA971EFCB87B8CAFC39ED2F195D3ED867
:1055C0009D6057197176C6F7F229E55AD34B1FF241
:1055D000FEAD1BB99BF1122B70F7AF65FD6C46A3B6
:1055E000E1BC893F2F7551E983573840EBB35F72B7
:1055F000E51F1B67BF173D67828AB59381404AF15B
:10560000A829C92D0F659EE7E70EB85F47A5098455
:10561000501050DDDB86D41284D3FB126CDD3024B5
:1056200095481FF213ADD15F28A2DD4A14CBCAA959
:105630001FF2FEADC25F28A2CD4A14DDCAA91FF237
:10564000FEADB75F28A2BD4A14AFCAA91FF2FEADD6
:10565000A35F28A29D4A14B1CAA91FF2FEAD5F0E36
:105660006BA75E6C0693D1AFA53EA916CB5C47A590
:1056700013711495CAA971EFEF8774CAFC39ED2F25
:1056800019613ED8BA6057193D76C6F7F229E51E72
:10569000F64B1FF2FEAD19B8DDF1CB36F77D1DA933
:1056A0001FF22AAD2BB8DDF1BEDA65A950DDC68642
:1056B000D86B26BE29A23F4B932DEB61A044DD653C
:1056C000A0CF84136CDD3AEFD1AFA53EB771BCBE5D
:1056D0000FF16CDD66FDD1AFA53EAB73AEBE0BF135
:1056E0006CDD66CBD1AFA53EA916405C47A5137112
:1056F0001417CAA971EFF487F6CAFC39ED2F191FE8
:105700003ED8BD605719B376C6F7F229F2E72CA947
:10571000543E5719F576C6F7F229E58A994B1FF2E0
:10572000FEADADB8DDF1BEDA4D2B50DDC686D86BCF
:10573000A4BE29A2274B93A3EB61A044DD655ECFF5
:1057400083136CDD3A6DD1AFA53EA916875C47A5E2
:10575000137114B5CAA971EF158754CAFC39ED2F1E
:1057600019813AA4833E8C6566CAA839ED2F198F3A
:1057700032A7833E8F6578CAA839ED2F199D33A6CD
:10578000833E8C658ACAA839DEDA6B89CED8F86088
:1057900057195876C9A2464B1508B74B1FF213ADDF
:1057A00020CFA313EEDA70A550DDDB86D86B3ABEAE
:1057B00029A25E4C9321EB61A044DD65DCCFF91397
:1057C0006CDD3AEBD1AFA53EA9167B5C47A5137102
:1057D0001437CAA9723EBC659BBE47A53F711439F8
:1057E000CAA97349BB65A5BE47A53F71140BCAA9D9
:1057F00071EF4D88FACAFC39ED2F191B37641FF27F
:10580000FEAD93486001E73017E937641FF2B49B9F
:105810009FE0C6F7F22993834263F0EF181601CF99
:1058200046A25DD974B581D9E0EE081583CED6A124
:10583000EDD904A331D970EE981532CB66A39DDB68
:10584000D4D301DB80F0C817C7CCD6A30DDB44DD71
:1058500091DBF0F03817A9CC46A47DDC54CE81DA78
:10586000112E5817A9E997C88A4A816ADFC8A13E54
:10587000CAD9E21ECB44EF4E8D89F68A9DBAE8D490
:105880007C5FA7205D688A17AAD8F18B521908BBE4
:10589000C9A4CE4D9507AF4D21F0B8898CCCBB156E
:1058A000ED2F194334A91FF2FEAD2DB8D0F16CDDF8
:1058B0004F99D1AFA53EA965B6CAFC39DF29155F5E
:1058C0007ED8705F6CB5D7AEC9F1EE29A55C4D48A6
:1058D00023746579F6BE79F16009A53B6EA9936DD5
:1058E000DCA4ECCA83396A29140FCAA9713E57197E
:1058F000457648612740EB34DAAD91F1B989EECCB9
:10590000B8156EDBF4014EDB0362546918BEE8F68D
:10591000487729F3A467C43E14B3E25FC8A2EFDA64
:10592000142050DDDB864086A9CFD8A2DD4A93BB88
:105930009461DBF2DA7CB6CFB116EEDA7E3850DD58
:10594000DB86C965D4BE47A5287105ABCEA91FF279
:1059500013ADD2BED9F16CDD4F715EA7243E3F6519
:105960008F70B112DFDA16F6D14895B0E3D460CA71
:10597000833948DD3682D1AFA53EB7660EBE0FF142
:105980006CDD66ABD1AFA53EB66CF9BE0FF16CDD38
:1059900066B9DED83560D916BD5C23F1CE29930BEC
:1059A000C972DC5F57196C76C9A2344A153C894824
:1059B0001FF213AD3BB8DDF1BEDA54BA50DDC68636
:1059C000C916065FD9A2234A935D9461A044DD65A0
:1059D000B0CF49126CDD3AFFD1AFA53EA916225CCB
:1059E00047A513718C024FA9F43E37B3145FC992D7
:1059F000E66CB6036CDE12EE39061A732B925F0961
:105A0000E5E1D1AFA53E5719BD76A3A565A7A44092
:105A1000B06972552047D45F47A5C87193893D632B
:105A2000E6206915D85C8B126CDDEF0357AE233E80
:105A30006C65D070B83D3E57762768A9D48C1AB1F2
:105A40008050982FA8292969EF65B16CFAA313BE7D
:105A5000CC3FEF75055BCF57713FAFB32D72291F58
:105A6000CF67F8836967D35F57190076B112DFDC1F
:105A700014709C481FF2B3AD8F5FC8A4DD4A477E07
:105A800050DD7B863F8607CD2612204A931934616C
:105A9000065FCA18CB5F8B126CDDEFB3AA4892F198
:105AA0009886605F47A5C87178A8DFDA505F8319D0
:105AB00061A88B126CDDEF9FDEDA93600B86B0CAB3
:105AC0002339DEDC11C79C481FF2B3AD4CCDC413A3
:105AD00067309733BAABDF8C1AB11A50982F4F2B1F
:105AE00034CFEF65B16CFAA34FBCC33FEF7505E14E
:105AF000CF57CB40B4B38772291FCF67081DB66755
:105B0000D35F57197B76D512E6581E140DA9336D55
:105B10007CA448CBA808E0581806A648A7E9CE10F0
:105B2000E25F47A5DD712126D646AA7DBC650C51F2
:105B30007A30D8DE66C2DC46A47D4186A8D1CAA0F0
:105B4000204A93D73461075FCA18255F8B126CDD3A
:105B5000EF79AB4892F1A8869A5F47A5C871795E44
:105B6000DFDA605F0B8668CA2339514A06FE614856
:105B7000FBF257E46B11A731773F477A50DD7B8604
:105B8000C918255C8B126CDDEFA1DEDAB7600B86DD
:105B90009ECA2339DEDC2E959C481FF2B3AD1ECD84
:105BA000E113204AF2482CA9543E57193E768B1235
:105BB0006CDDEF9BDEDAF1600B86B4CA2339DEDCE4
:105BC00066C39C481FF2B3AD48CD8413204AF3232B
:105BD0002CA9573E571944768B12C037F73D1CA9A4
:105BE0001FF2DBAD265F47A5C8710578F44BD35F84
:105BF00057199876C9A4094B47F850DD7B86C91818
:105C0000AC5C8B12CB33F7E71DA91FF2DBADCC5F89
:105C100047A5C8718D3A9C481FF2B3AD8CCF8E1347
:105C20006760A6D7CED8D960D29CDBAE49A4254BFD
:105C300005A2964B21F0FF8728CCFC136EDB413D7B
:105C40004EDBCC605917FE5C59A3154B95DFE04B3A
:105C500021F0068744CCF3136EDB3E594EDBD16056
:105C60005917DD5C48F15F0985899C481FF2B3AD87
:105C7000F0CD8013204A93E3346191F11387BC5F28
:105C800047A5C8711514954B9A7562750CCD821392
:105C90005F29479250DD7B86C918565C8B12C2364D
:105CA000F7411DA91FF2DBAD6A5F25FFD029CB4F5D
:105CB00050DDA3860B86085F2670DD98C85D50DD39
:105CC000A3861786C5C82400D029C82B0EA91FF2A9
:105CD00053C1D2C918010B383739A04842F4CC65FA
:105CE000E1CE44A3DF9966105FA9D35F571991767F
:105CF000D9A4454B0566B84BD35F57198376D9A411
:105D0000474B0590B64BD35F57197576D9A4494BCD
:105D10000582B44BD35F57197276C9A45E4C471EF7
:105D200050DD7B86C918965C8B126CDDEF05DEDAE0
:105D3000C2600B8655BE3AF1A12993AFCC61D35F07
:105D4000AB7030BE0AF16CDD17619C481FF2B3AD39
:105D5000D0CD4D14204A93C3346191F14587DD6E57
:105D60005101E02905F6A24B035F37DC9311D9926C
:105D7000504A05F2C65EFA52D26CE8BE47A5455DB0
:105D80000C6450DD5E8849A8B9AAD9A2064B051E4D
:105D9000A94CA97572751EB0DAF16CDDB0A51A892F
:105DA00021F0CD8BAACA4642E730174B50DDF8727E
:105DB0005646BCCA773AE73017593C641FF2B49B89
:105DC000C59FC8F56CDDD2ED50DD0D81484549B861
:105DD00047A5AB739341336E0A1ED069D2CA043B08
:105DE0006CDD17F9AD89D35F57198076C9A45A4B7A
:105DF00077F0B01E10AD69060A5FD99287608E0FEA
:105E0000BB89948E5175E49EC0F8F02993993E5F4A
:105E10009A45DB651ACAAE25DEDA811950DD748831
:105E2000CD6BB2BE47A56E8193BD4E58E01EC96AC8
:105E30003ECA043BE12905A4D94FD91E5719F27E69
:105E40008CD1204A93D12161035F37DCB311799261
:105E5000504AA5D26C5E1A4EC94554CADB16E730CB
:105E6000178150DDF872CB691D9E8B126CDD0447E3
:105E7000CEDAFA5FC9189E5F8B126CDD0455CEDA5C
:105E8000FC5FC9186E5F8B126CDD04A3CEDC92F34D
:105E9000E8D402CDA412DEDC71989C481FF2C8AD94
:105EA00030CD3212DEDCFFA69C481FF2C8AD3ECDDD
:105EB000DD12DEDC18B450DDE56CD1454E5FA7681D
:105EC0005D980542D3791A4E9145085F47A5C87180
:105ED0000542174A113E0B86D6CA3639DA4A47DEE2
:105EE00050DD9086F5866671FE126CDDF1CC5116A0
:105EF000148ED27C77BA67D1504A73ACA10691DF79
:105F0000CBB55BAB8B126CDDEF215666D35F5719B7
:105F10007A762140DE789383197199815279489E6F
:105F2000CDF6760993B12B4B9E424C4522CA0B13FA
:105F3000EB2F93A713631FF28A86729EBB124CA0AD
:105F4000840EDEC8928E92798A5F47A5C87193DB72
:105F50006F58964257191B7470D16CDDC3746889F1
:105F60009A42C918145A59A34F4D95F9314D21F051
:105F70003B89DCBFA33F00297F57E3AEBC8CFC65A7
:105F80003B7042F9712908679667085FCA161FCFF0
:105F900036126CDD4FBDAB4892EFDA16C35F47A5F2
:105FA00028717DA2DEC8A2DF4915605C4BD1F3DE0B
:105FB0000C2454DDF3555719727683A564A8A4F018
:105FC00092692A55D86B52BE47A57A73945D51D910
:105FD00020EE28161BCF56A26DDA844BB1D9F0EE15
:105FE00018155DCEE6A1FDD9147921D980EEA8154A
:105FF000BFCE76A18DD98D6241DAE0F12818F0CAC2
:10600000E13AE66C8EF1358991EF438A847DC805CB
:106010003EDAFB16AEA9FAB643D49ADFC7448F3DE9
:1060200093B5DA60923EC918D25B4BD16CDD8F0517
:10603000DED80B63CAB5CFAA47A50672080D86B98C
:106040001FF2CDAE9C7147A5E2724D64DEDA0C639F
:1060500061B44F5147A5E2729D4EBFBCD296197AEA
:10606000B0CDB4166EDB03614EDB0D6359171158CA
:10607000CBF1DEDC7F70DED80B63CBB5FDAB89A244
:10608000594E9317F6603D8D79651ABE6128975079
:10609000C9617B891FF2CDAEF071C500F329930B66
:1060A000EB6191EFC78B2A49E1041EDA04AB50DDA6
:1060B0009587119CE5AAC9A22D4A14C6DEDAE05FD5
:1060C000D57457BE47A57C75870950DD4F87591792
:1060D0002A5B4CD16CDDC3FE4EDB0B63155401CF44
:1060E00086A27DDA8D7091DBF0F0381713CC29A2EF
:1060F000AF4DF5620C4D9985C0827ACBD1406CDDF5
:10610000E63B7ED81B607916035C09A26A4BD59EDC
:10611000534B1FF25EC07D5F3512BEDADA192ED8FE
:106120006762D1AC53A3C9A6F67893BF3F7331EF32
:10613000578702CF46139EDA953B0ED82260571937
:106140005565D2120A4A4C46E8481FF2A7BE40CA1B
:10615000674B3A4A5054CEDAEE5FC918805FB6A159
:106160004DD964F391D919F31817B5CCA6A35DDB0B
:1061700054E281DA71EF9A8908CF1B15E670FC8230
:10618000DEDCA98D5719E76469A25C4AB51CA148F9
:1061900051EF4987C4CF48136CDD9AA035488D5F15
:1061A000A916F15A39A2B24D0D8E29B491F3E1B47A
:1061B000BECA284B2C38565704D85BEF831694CFB1
:1061C00047A5738420C4F248D85FFF86C2CA144A28
:1061D000C94A01D23ED86662B9168C5AC138D54632
:1061E0000574C6661FF2AABFC0DB7096A8CEE06A2F
:1061F00050DD2699E4865A5F8E12144A9369007026
:106200001FF277BFD85F8212EEDC660ADEDAF15F3A
:106210002816DDCFB6A14DD9648991D919F3B817E5
:106220005FCCC6A3FDDB34B5E1DBE0F02817C1CCC1
:10623000B6A36DDCA4A691DAF0F126A955BF2F3FD5
:10624000CF75FEA39967928A296DD470A8F10C7757
:10625000367DDE89FE8A48A9BEC2A91245E555529F
:10626000A8D5E16B5AA9AA069760E9CA0C6C591126
:106270002EADD1A84DAF8712564AE5F250DD105F22
:10628000D20618DFB11280CE81887DCA1FF24697F0
:1062900079DFB39274CB0506DA4F9981E279665FB4
:1062A000CDBAF7700C58CEDCAD5F6B949F411AF1FC
:1062B000E6581EAC04DCF255CB94294147A5598120
:1062C0001E46D6CE095FC9063F5FAF685798054C9A
:1062D000A648A4DF30861A5194305C4A688AA70623
:1062E0009AFD0986F57AD894DECC83EAB31F0AAD0D
:1062F0005A07E2DC8E1211290DF6C756CBF32A7C21
:106300008E47D61A5A4A6C51A70631EF12872ADDFA
:10631000CB66F79881149ACB31EFCD8B3E7D680523
:10632000BE34F9C350DD2264D786270D506021A00A
:106330005E7E76C84ADF77B6095B59058C2AB5DFE1
:106340001EA9613E0E86F25F47A53E847D4C6FCA52
:1063500031E11C19D4CF1612365F8DAF258621F09E
:10636000138B72CC80176EDB516F4EDBDC64C91669
:10637000075FC134E73905E6F7489981B275FECF6A
:10638000E313E079DE75DED89E60D1A8B5AAC8F126
:10639000EEDA8990C76A2A52C9659B9EC8F1DEDC95
:1063A00052A77ED8C2607965615FC120F768D84F77
:1063B0007C46447DA31A57A9CB20F1689329A57187
:1063C000A1F1188B44CD87177EDA35C96EA9DA5F43
:1063D000D1944B413AF18058B8C624DCF255CB94A5
:1063E000734147A55981A576904F41EF188BC6514F
:1063F00070308EDC56F37EDAE164C916575CD9F151
:106400006CDD803BCEDA9264C9188A58C9A2284B49
:1064100093857F6B1FF2279B98CFE0136CDDCD0D2A
:10642000DED8B86057192557C9F1EE2993B98A47C4
:106430001FF2D0893ACAFD16DEDA853AD66A224EB4
:106440005719375CC8F1DEDC094F50DD5B5F281659
:106450009FCF56A26DDA84C7B1D9F0EE1815E1CE00
:10646000E6A1FDD914F521D980EE511AC4CBC0F8AC
:10647000F029F49C50DD7C74C916D35C47A5A65B5B
:10648000FD1550DD506557194C5FC9A2064B931B93
:106490005B601FF2689698CA5C126CDD0C9950DD47
:1064A000086C5719527A47A5124E053A9148915BEC
:1064B000564532CF8513E66C9E4D50DD7E85511AD0
:1064C000CECA25366CDD15CF50DD208F511AEECFA8
:1064D000CC178EDA0BD397487B3EB965D2CADE4C17
:1064E000DEDC70E5711650AD79186C5869A4E34F85
:1064F0009365FE6D1FF2908EF6CAB5403EDA70F9D4
:10650000AEA900B747D486DFC1417F3D93990248C9
:106510001FF2C59698BCD8F16CDDB02356DC91EF24
:10652000F387A06E4001A40912C1CFA91FF22687EC
:106530008C5FC9A27E4B15A67F4BA85D4C45AECBA8
:10654000C8A6FD98A5D48E4F41EF1A8B0CBFC94148
:10655000F25011A776524A697918855869A43C4FC0
:1065600097774D4F2D53C916A658D9A22D4FAD7808
:10657000674EDD525F4536BE19F3A064D8761652D9
:106580006A6999185B5809A43C4FDC74518991EFF2
:10659000178B02CF8617EEDE060CC1069575DE8CD2
:1065A000B4AAC8F162099535BE4F2A1ECB652ECD1F
:1065B000A91773090524D34B99818A75DCCFDA12A8
:1065C000CEDA19C22EDC72F3C8D4C39EC9A2624CC3
:1065D0000DF21FB99E46DA65D6CA94131A4A50DEE8
:1065E00050DDE56C511A69CCD6A30DDB447F91DBFD
:1065F000F0F038170BCC46A47DDC546881DAF98CB6
:1066000048A9955F6B2091687E08BA1B0FAD4906BB
:1066100001DF0E1201290D1BC755BBF32A7CE75F72
:10662000A11E57667272A20691E3DA0A2445501C35
:10663000574A7361A70691DFDA06825F212CD7548F
:1066400096C25ECA91EF1287C07D1801424A535626
:106650008140D8B422D4985F47A54E4EF2DC20C8C2
:10666000FC5FCB6505663118723945838CA9685F7C
:10667000F391C942E1FE28772B998467DB6A24A154
:10668000385FC138D5460512C666085F2FDC771122
:1066900069928E29C5750EA91FF2C1C0405F821292
:1066A00041293A36F9DCA8F3D01A40CB9808544A6D
:1066B000C5300FC85979A290065FB4001E8164B836
:1066C0004ABD7146C674315FAE695B980B4CCEA96A
:1066D00079FDD986BDC1791ED6E8B5D64F6DCB5FA1
:1066E000ABA09155BC124B9F7EA62FCA71E10D86BF
:1066F0007E47D61AE09E1EB850DD0163281631CFC2
:1067000056A26DDA8495B1D9F0EE1815B3CEE6A194
:10671000FDD9148356DC50F0981745CC26A3DDDB59
:1067200014B3C1DBC0F00817E7CC96A34DDB84BDE2
:1067300051DA30F11818E9CD84C83C00ADAA51FFF8
:1067400009F227444BE084D09677ED65296D045F0C
:106750003794AD41961201A14116C14833BC86D48D
:106760000DCF35A2374A12F6C2D822F5B1A017557F
:106770003594C9CC7874B8120DAD410C93DDC99233
:10678000F14A88637C46447D531A6BA977948BCC7D
:10679000389039118EADC308F1DDC134673D805F9B
:1067A0002CA94874FA7920B4D8F16CDD46AF1248B0
:1067B000A1F1158B34CD8217DEDA52BDD66A1A529A
:1067C000CA45A2CF8017CEDA4FCF9A481FF2E29384
:1067D000D79EC8F1965FB623D3A1A23E57191F5C7E
:1067E0000512CE090902CFA91FF20A87705FD9A44A
:1067F000284F0560974F91EEC6886ACE3714DEDACF
:106800006507D66A9252C916D05FC9456639DFCF8F
:10681000DED88D5FD9166B5FCB2CF154158E2348D3
:1068200091F1C5866B9E29A2294FF5BA924F81F34B
:10683000AA1A4D1180126CDD1E373ED89164B9162C
:10684000C15847A54681F146DED8F164CAB587AB89
:1068500049A23C4F95C4814F51EE178B0CCE861741
:10686000124A0D4429B491F3E1B4F25F0D38954614
:10687000C5E40A661FF2C1C0335F15124C6D5C831C
:10688000BEDD0F8A118691A14AD1EEDE0618C1063F
:10689000A35F71A0AD550D389546C50E0A66D85F49
:1068A000FF86ACCA314CC656FEB4D454AC7BDB86F2
:1068B000F4797E0E9EDED99850DDF199CBB32D7020
:1068C00048D1A44A78C4B046107D35E13011C99250
:1068D000EFCA59D2F652CA691686C0485217A23971
:1068E00026019467E28A491CD9AA85353B6D882F19
:1068F000926DDBF225B1C57E7801BEDA05FB2ED89C
:1069000092645719EC6649A8473A410AE6A9928E63
:10691000E48C06AE29F1D6296DF63E798F655D7956
:1069200040BE3100EB2D18C750DDA96E560630DF92
:106930004F2A755215A0DFDCB0ADE586855FC13802
:10694000D54605D6C666BADF030693C865A28E296A
:10695000C5B10EA91FF2C1C0845F82129EDA4F5DDD
:106960007AA9413E6DA057574DD113DE2CF8C9DCF2
:1069700098F3731AA6A9FF12C658FE649648A0B3EE
:10698000E5D4859EC492FCCA0B90C940A0B3E5D45F
:10699000265F47A54E4E28961A46667D4386730DA0
:1069A000B0607ECAB624D66EAA85CBA03F55A2920F
:1069B0005ACA6DA4A74E3D4E1886944976186A3D72
:1069C0004EC0D44819B062D4545FF012E670FC3265
:1069D000DEDCA98D43863509B0607ECAB65C1EA98F
:1069E000613E57199C659512294A6A0BEBDCB8F396
:1069F000E01A75CBA3A62F407DF8CFCA91E13606E9
:106A0000FEDFAF2A55526752A70656DE9F0559A0F2
:106A10004DD1AEDDC6810F4164F2CC861A095060BB
:106A20005B2BD435AFA970645179519E2B124C6DFC
:106A30008415F7C8CBDFB51648BEC9F1EE29A5D637
:106A400061AC523E996548CA314CA94AE14C99481B
:106A5000C75FF086C25F47A5D684205AF248D65F4A
:106A6000FD866CCAF74C564AA5EAF7C8CBDF5C1B1B
:106A7000FCCF5AA8514A7378A156F4B542D456C1F6
:106A8000D9126F6DB6067ECA9A3FD965E4C0B912B5
:106A9000C7E7759E26D7016B5AA97606B7605FCA0D
:106AA0009720EC487DB0BAC519BE2443D950955FF4
:106AB00032AB823EC96526BEA09258CA6DEAA106D5
:106AC00031DF796584BE19F16CDDFDF072AB423EB9
:106AD000896582BE47A51C847DD878CA3A3F79650E
:106AE00082C08912C1E715EA2CD7A16B5AA96206A8
:106AF000D7605029C4E31FB9045F37940341AB6FDB
:106B00005B98E5822FC8131EA9657ABE47A5B44DD0
:106B10003490E6CC9DEFD1A801AFCA3E6CDD6B3E50
:106B20004189FADF4306A6DF9112EADC18ACAD48D2
:106B3000FF6D48A4D709B060E7E8453A4F6DA2E180
:106B4000C908CBBFD9F1C6E7754837D7016BC12358
:106B5000A05358354AA183185FC903DF29B248DC26
:106B600061A76DFF7DF180F6201C1644B3CF86A28D
:106B70007DDA94E2A1D900EE2815B5CEF6A10DD9A3
:106B80002411D1D990EEB815D7CE06A19DD98D1A72
:106B900091DBF0F0381769CC56A42DDC640E7ED85A
:106BA0009664791622588012C829F54B50DDA899B1
:106BB000C918595866709D98B52AD84F31F1CE8BB7
:106BC000CECAE935DEDA15C6D66A1A52A845AECF66
:106BD0001A15CEDAD9D1D66E885BC91A447147A589
:106BE000BF83A5724C4B41EF5C87AACF5D13AEDA31
:106BF0009AF350DD2699B486845F29A2AF4DF56ED5
:106C00000C4D9985C08286CBD1406CDDE6377ED8AD
:106C100027607916035C09A2764BD58A474B1FF291
:106C20005EC0B95FE512254A3B2850DD6E97B486F9
:106C30004C5F29A2B34DF5A6084D9985C082BECB05
:106C4000D1406CDDE67F7ED82B607916575C09A2B7
:106C50007A4BD5C2434B1FF25EC0C15FE512254A95
:106C60003B6050DD6E97571946649512294A15FC12
:106C7000814891F12786F7BE47A5517BE5ECCB4FC4
:106C800081EFDF8B09B6D8F16CDDA08FDED8DE6432
:106C9000D1A8D3AF47A5D179057950DD0490571914
:106CA000146ECBF16CDD78953ED8A864B9163658D1
:106CB000C9A2F14F1524CA4F1FF2E293005FCDF82D
:106CC000EF299357454D71EFDC8BBACFDD17CEDE40
:106CD000E644210691EFE08B48CFD1176CDD1ED141
:106CE000E2482F1EC916915FC134C73993792D79B7
:106CF000913E5719076C29A2F14FF56ACA4F954585
:106D0000DA650CCA5215DEDA2E08D66A7A4E5719A1
:106D1000A46ECBF16CDD78253ED8A864B9168658F0
:106D2000CFFBEF2993B1454D1FF2908ECCCFA21728
:106D30004E29746AA00691DFD4B563AA47A5ED7BFE
:106D400093D5C14B91EFD08BCB6EC8066CDD8F4CC9
:106D50007389958E2A79459E68408E29B1C2AE48C6
:106D60003EFD399258C1B91E6F6D7133A00694DF94
:106D7000D1A86BAEC8406CDD104A4116141E59658F
:106D800049BF99F1DEDAE486465E415158450C6E02
:106D900050056CDD39895489998E8A7992CAFC151F
:106DA0006CDDE1A250DD8D6F5719567196A22DDA78
:106DB000A420A1D900EE281577CE41A6CDDB042D65
:106DC000D1DBB0F0F81779CC86A33DDB745FA1DB93
:106DD00030F118180BCDA512994A934F0D4891EF39
:106DE000D48672CFC51286CABE68DC46A47DD91887
:106DF0001258C9A43F4F0566FA48A1EFEE86D4DFCA
:106E00007292E058181ACEDAF564C918EF58C9A280
:106E10001B4A1582E0483DDF86069851DA30EEDCE9
:106E20006B27DEDAF664CA65A8CDAE172A6D620B51
:106E30009EA9E13E92669270F83DB2290A13CF6591
:106E40008F1E5719236C59F1B2096665A16DFBFAC3
:106E50003986B9C2B91E58E575544F6DFDB647D491
:106E6000E3DFC134673DC9A78948BB6D04A4C10FE6
:106E7000F06085D2B5F8D3D8ADEF5A1C5445701CDC
:106E8000274ABC7C5A899985E2AC0845DA1CE0792E
:106E90001694D2B9DA5FFD8696CAE24C705F989973
:106EA00042BD923ED965A49EC600FD3820AC764610
:106EB0004A7D096564BEA3ADFE4A70270E440BFAF5
:106EC0009992D37A0569BC98142670754965A575A1
:106ED000195F6A448F4E9927DCAAA13EAFACA9790D
:106EE000212CD75487253CAA813E1386E2CA52152D
:106EF0007DA805620148297551795D91A8F652294E
:106F0000A8E15A89D13E1965290E38027EE0E6FED5
:106F10001EC842DF7B1B9271DA40F54888DDCEDC6B
:106F200092F3E8D4A16FD816CA4073E44EDBF8643C
:106F30005719785FC8F168098DAD9F55E27A0F99AE
:106F4000975A4001DC1895D5B94F913E281681CF4C
:106F500056A25DD974C581D9E0EE0815F3CED6A14D
:106F6000EDD904F331D919F36A1BEBBE84433650D3
:106F70009D82828630F0581777E846A36F6D14EC37
:106F8000C1DA91EF328B16CFA3175FDF151EB44F16
:106F900091F1328B0BCFC6A26DD9942551D930EE29
:106FA000611A22CF5012DF79465D61FE09F26F3A15
:106FB000F0CFA017AEDA6FB1DC66A13EF120BB9E28
:106FC0000670BD981A50D9DC171EAF3A59CBCEA621
:106FD000C0608D27DFDC501D574545E9B1A5E4FEB3
:106FE000C570B74F61EF338B40C54DD1ED88961F0B
:106FF000111670ADE84496BE39F1D478EAD20A662B
:10700000558591945543282ECF66859BB64F151E06
:10701000BF1A75CB1EA6A5DE8F8D8CBEDB5F511A05
:107020002FCD56A42DDC64B4B2481FF21ABCA25F67
:1070300042D16CDD5602DE52A2696C65B460DB1889
:107040007639A6D456182DAD691CD3A996A22DDA8F
:10705000A4C051D819F3D194C141C120F76886C8A2
:10706000AFBE19F3C9167F5FC841873D078DDEDAD1
:10707000715FCC65709EC1F1DEDCE57ADFA991F12C
:10708000318B02CF2711DFA9051A304919F3ABB5AF
:1070900098AE09D1467866C7BA79D1523965415F51
:1070A000E46F1A981134D66ABA53D0364905B760DE
:1070B000EECA0E98D9F091DFE136DC7D5001F6740E
:1070C0001D78788991F3D2A840E76BD1DE7ABE3B78
:1070D0000AD377815A758AC452D1BAE19E1DDF78EE
:1070E0004A52991F827D5801BDE3972B01D1211E81
:1070F000CBB6CBAA69ABC46C960976D31A1E711DA8
:10710000079EC943A73DEB244FB96BF84A4554C6C7
:10711000C8F166DE05F556DC913E511A9C3AC9A4C9
:10712000DA490CCFDEDA8B5EC916505ECF0E5A18E4
:1071300005A02649A1EFC285017169F1EE29071466
:10714000CD6219F3F817F9CC86A33DDB74DFA1DB20
:1071500020F168189BCD96A4367893CFD071E04D7E
:10716000496572BEE33508DD3F45926DEE82BF860C
:10717000FD7147A5EC812176D45CAC635179225F27
:107180004B2871508D71D748BA5FA965FCBE8D1F21
:1071900033676B8DA957D2AEA27C1ABE8127E12C32
:1071A0005DA7DEA9F964C965505879016862A0A697
:1071B000DFA91F8F5A8ABEAEC9F13DDA542C41D8DF
:1071C00020EF48152BCE96A12DD9445BF1D919F3A8
:1071D000B19CAB595505E4641CD256DC33857CACBC
:1071E000C6457E1CE06018E042BD976DE0A4E6CB8A
:1071F000C9F1EE298D60F46EA85BE91A467167F15A
:10720000E6581E1CF456CC7D731ADBA9F5122B4AE6
:10721000A5F060A9513E996516CAA94C274A8D8AE6
:10722000C248CA5FD1AC51A3C9A6F678A5CC60A963
:10723000513E99653ACA314C094A413AB0A986F3A0
:10724000B01A15CB0EA648DE56BE944819F318188E
:107250008FCD8DF82F2953563EA91FF27887905F66
:1072600000A7BF2993F1714BDF5F0B1B0EBE47A533
:107270008D4B64E291D819F3CA6CE8BE29F16CDD3C
:10728000AA92D7AFA33EAA6586CA6C24E02F176FD7
:1072900050DD4271511A13B8DAF1C238F67D50DD73
:1072A0000D6DD66937BE29F1D629933FA24619F351
:1072B0005719846C47A5267E82760E11CC85F3ACD7
:1072C000CE8E3CD2C41AB5373598314E7A79516199
:1072D00058057C3DE01450BDF1F330808D9FA040F7
:1072E000D51A0510E45E7365BC8C6E59DC187639CE
:1072F000F605C0BCA01F577918CB423F187825D29D
:107300005548CA5FD9860A5F8312FE4A9629A16E44
:107310006A79E2754D611905AE87EDEA445F019E19
:10732000EBB401717D40A270DD76AD8657F3801A13
:1073300017CBEEA64E89D8A297BE8F52689B845574
:107340002B1CD154094EE4B9A2AEEA75B351F23008
:10735000C468FC4CD656D3555745E0512B30D16804
:10736000097E16BD98F3C01A0FCBFEA655DE23503A
:1073700056B9C42DDC1AFE514101F7707372C9DC95
:1073800098F3511A5D8E4105DF298D1E5299201FF9
:107390005056D2AEB7E18E39A66D01762A4E3945E8
:1073A000F14F70D251099976C6BAAA811278FB7D45
:1073B000F804F364DABEE56EBB85AB9CCF59CD18FB
:1073C0009639249C0106336D7CA48E41E330073C42
:1073D000B80150674B4E296DE88ED861AE896B4A73
:1073E0005E55DB55725518716EE1C458FCF2D656E5
:1073F000CC7D6F9CC35901180950351357B9CC691E
:10740000C9B2BD5FB638F1A1E44674B9AF9D9A8A9E
:1074100078AEFFD15E0AE428B2BAA99C257898CB51
:107420003EA6C5DE3CB0A9DCB0BD127CA451D82E6E
:10743000F4DE0CA6C9B019F32A655C513E30E6684B
:10744000405E3C5E8465CD8CF2596901C064F844AD
:10745000DA42CB6937A4DEA9A9A666DE898D36DDBE
:10746000C26F22456CCBF5E1E639243CCEB9CA8D1A
:10747000E2ACC50FE9012F39EB762956997DE2A4DC
:107480009AAEF3A627409747EF79924E0C553FBE30
:1074900041A61E09ECBA2666998501E4A5AEF05016
:1074A0002A3C0B3629DC78F3FC1A73A97705EEDE4B
:1074B00005242EDC72F3C8D43711D66066DE6D2B3E
:1074C0005789A859877956CBC9A6CEDEE65821063A
:1074D000A0ADE8D44D7DE00157781B32E56EA4F3F2
:1074E0003F1A65CB3EA6C5DE3C7CAF58092D4379DB
:1074F0004B515805BE48A037311690ADD8D4611114
:107500005FD1E66C96F5C8A0221EC0A82DAED7F9B3
:10751000E578FB3C5B897781BA758CB6CF40CE2984
:10752000E5C174B9ABF3AF945F41C13038400D2071
:10753000C8DC98F3E07E3ECBD0205E51DA32F442D4
:10754000F146477452485E1746507E4C9EB92374EC
:107550005C8BB659BC18F639E7422D429569DE902E
:1075600059AA4337BF39A84C7A6236896A7966CB03
:107570004337673D2635F8DCA04DCAA2FD4341A63E
:10758000F54224E4DEA1813EA96582CBD600DE353A
:107590008D045E6D1BF25F9B8F585117674F8D0AEC
:1075A0005E6D1BF25B9BB5585D17634F8D38576757
:1075B00014F24991A5AAC134B03940B41EBDD08996
:1075C0005A79A2A14DD1CDA80486D106B0AD511AE9
:1075D00087A3D969A258DAC807B9709DBA7599CB43
:1075E000C120F5441EFA3FB9B09DC2756BCB41A6D0
:1075F000705F98F54A4F667D3B54BCCBB8F0660986
:107600009B17494F2964E2A4F991CFA6CF4EE60A11
:1076100056DD19F33119AD792F38D570501CC9B02A
:1076200019F3D3642CAAC60066DE90FB9E86C23D89
:10763000717584815101F36C8EC9FC86B82D5AA9ED
:10764000AA918FF0FE3C1AD88FBAA66D99651B419E
:107650002BB04E4AF7CAE56E016BFAA23FC1E33880
:107660004E56367EF45675FDAFACDA53E82EC4683C
:1076700007EE7C6EC16BEAA21A413AB00E56266242
:107680003C5694FDE992E7436B30D2E8B8AAFE4439
:10769000727B6CA410C1291E7F6607B428667B8D9F
:1076A0005AA93D091951E8396659D66A5B4E379493
:1076B0004F41F230C468FCA8D656A2AE99C517A9AE
:1076C000D750AF4EF5350286B72DA8C420ADD14FA7
:1076D0003A3C0B4629DC78F3001A2DCBAEA6FDA868
:1076E0004616A062996DDAA27ECBCEA6F5428D7ABF
:1076F0003CD6E15FBC24065FCBB03E5676E03AD67E
:10770000F16B3AA296C1B91EE1E875062AD6016B63
:10771000AE24E253D038D0E83514BF540A7DAC24EF
:107720009053A82E5768422691482282511A8445C8
:10773000F22CAF2A8CF5F456CC7DEF9C8B59590175
:1077400004643C48D656AA7DA31AE3A9C9A6EEDE76
:107750004150934819F3E08051704E376819FCA2EC
:107760005A99F63D4F55667E5305CEDEE6F8210662
:1077700019F33F7CE4CBC8A6FD988DEEFFAB2B8CB4
:10778000F3A03945B4126B092F96E556FF7D48A446
:107790003249FA1842507A907EB9B379FC907A5502
:1077A000BC1CC468FCBAD656AA7D6319C5A929A613
:1077B000CEDE0526CEDCAC5FF586075F861266DE80
:1077C0001C3A5767168457559FA34DE135288F1FE4
:1077D0005E554952991A96CB79A67FDEC49211065E
:1077E00070AD511A12A9D9A6DEDEF57E3FDC90AD50
:1077F000D8D46D1141A64C5884E65BD905EF29B267
:1078000009CAB2123A4A87C75BD91EF08AD55E1EF2
:10781000910866DE80148248151ED6161DCEC92A30
:107820007F3DC6730E09D955D1A0B35541A63A4A3A
:107830005030A2480AF747543E9EBBCE3F067DA576
:107840006FDF11125617070E195116408DD8824856
:10785000DC5F4C4579CF47A59085C60B0E09E155F5
:10786000511A4471B0AA5C18A4D3CCF4921B69429B
:107870007FE8B1A558E37EED51F712F4511A86CA9C
:02788000B6E070
:107882005F4986855E49115E49858D5E49115E4973
:1078920085935FB6905E4985A1A149115E49EAB31D
:1078A2004C5A8F70EA97A85E4911C55BE7BC035A30
:1078B2009E70BA87DF5C2B135E4985BD365A79719B
:1078C200B198AC4D21127C1585EBA14B12664D8609
:1078D200D25D4B1760B1EED9BF49A75E9405C55C76
:0C78E2004813684F88E35B42195F528531
:1079AA000429DBC19CEDDB1A2AC5D7B202F02F14D9
:1079BA00EEFBC6160443009D8FD9291655158A9EDB
:1079CA00EA3926642FBDACF84733713BB1B903518C
:1079DA003D7A2BA6B00A5844811FA3B40E5C478394
:1079EA0014A0B70F5B46820DA2B20B57427D0FABB4
:1079FA00BD0450397411B2A3FA452E68E78194EC9C
:107A0A00372059DF8E84DC260F48D4E0F2C913FBF5
:107A1A0035B6F4EEB5FFE720BACBDBA0E9D10AAB65
:107A2A0021358AD4BCF45C372F74BEA6DF600A18ED
:107A3A005FAA92CB7D1E774C967FB87470653B85A2
:107A4A006EA86D41542C77609A474C59206C55901A
:107A5A0050574E17634E89625C4B125F4A85685EC7
:107A6A0049115E49866E5F4B13614D8A73584E1AEF
:107A7A0068549173515923725E9C9D4554307F6CB2
:107A8A00AAAC74653F8F7CBBAA657751A18FCED50E
:107A9A00101865B5A3E2C03D2F7ACAB8F8D12735C8
:00000001FF
